S01700006D6170735F626F6F746C6F616465722E73726563D2
S113000008E1FF1F11040000EB040000C1300000F0
S1130010C3300000C5300000C730000000000000FD
S1130020000000000000000000000000EB040000DD
S1130030EB04000000000000EB0400005F0C000073
S1130040DF820000DF820000DF820000DF82000028
S1130050DF820000DF820000DF820000DF82000018
S1130060DF820000DF820000DF820000DF82000008
S1130070DF820000DF820000DF820000DF820000F8
S1130080DF820000DF820000DF820000DF820000E8
S1130090DF820000DF820000DF820000DF820000D8
S11300A05D5A0000615A0000DD320000E1320000B8
S11300B0DF820000DF820000DF8200003968000078
S11300C0DF82000045680000DF82000061680000F4
S11300D0DF820000DF820000DF820000DF82000098
S11300E0DF820000DF820000DF820000DF82000088
S11300F0DF820000DF820000DF820000DF82000078
S1130100DF820000DF820000DF820000DF82000067
S1130110DF8200007F7E0000DF820000DF820000BB
S1130120DF820000DF820000DF820000DF82000047
S1130130DF820000DF820000DF820000B50D0000D6
S1130140DF820000DF820000DF820000DF82000027
S1130150DF820000DF820000DF820000DF82000017
S1130160DF820000DF820000DF820000193A000015
S11301701B3A00001F3A0000DF820000DF8200000B
S1130180233A0000DF820000DF820000DF820000EB
S1130190DF820000DF820000DF820000DF820000D7
S11301A0DF820000DF820000DF820000DF820000C7
S11301B0DF820000DF820000293A00002B3A0000B1
S11301C0313A0000DF820000DF820000333A000091
S11301D0DF820000DF820000DF820000DF82000097
S11301E0DF820000DF820000DF820000DF82000087
S11301F0DF820000DF820000DF820000DF82000077
S1130200DF820000DF820000DF820000DF82000066
S1130400FFFFFFFFFFFFFFFFFFFFFFFFFEFFFFFFF9
S113041072B60E480E49886000220023002400258D
S113042000260027B846B946BA46BB46BC4609482A
S1130430854609488047094880470948804762B68D
S113044000200021074A9047FEE70000000000005A
S113045000ED00E008E1FF1FBD6B0000FD29000076
S1130460432A0000112300000000000000000000E7
S1130470002A01D101207047F0B41F46034603242B
S11304802340002B09D00424E31A0170013008240E
S1130490E141521E26D05B1EF7D1042A1ADB13D089
S11304A0002F11D00C460D460E46102A02DB72C0F6
S11304B0103AFAE70C2A02DB32C00C3AFAE7082AAF
S11304C002DB12C0083AFAE7042A03DB01600430B5
S11304D0121FF9E7002A05D0017001300824E14118
S11304E0521EF7D1F0BC00207047FEE769140000EB
S11304F0000000007B140000000000001115000043
S11305005F160000FF14000083150000331700007D
S113051000000000D117000000000000B514000026
S1130520000000008F14000083150000471700002E
S113053000000000B1170000000000001F140000BC
S113054000000000E91400000000000000000000AA
S113055000000000E5170000000000000B18000078
S113056000000000471800005F16000000000000B3
S1130570000000000000000000000000000102462E
S11305804D230000DB23000000000000F9230000DD
S1130590872400004326000073260000D5260000AF
S11305A0E126000069270000712800000000000017
S11305B00D250000FF25000053250000A1230000A5
S11305C0ED27000000000000000000000000000013
S11305D00000000000000000B9820000C382000097
S11305E0CD8200000000000000000000A1310000E6
S11305F0E33100003B320000000000000000000076
S11306006F320000E9190000191A0000591A00009D
S11306103F1B000000000000791B0000673500004C
S1130620573700007737000000000000000000008A
S11306309F370000C55A0000075B0000E95B00001B
S11306400000000000000000155C0000072F0000FF
S1130650912D0000B92D0000352E0000712E0000F0
S1130660F52D000052656164790D0A005472616EC3
S11306707366657272696E670D0A00005375636371
S11306806573730D0A0000004661696C7572650D2F
S11306900A000000EB3C904D5357494E342E310074
S11306A002010100022000FF7FF080000100010030
S11306B001000000FF7F0000000029313233344B79
S11306C0696E65746973205553420000F0FFFFFFA3
S11306D0FFFFFFFFFFFFFFFFFFFF000046534C201B
S11306E04C6F616465722008000000000000000087
S11306F0000000602C42000000000000412E006653
S1130700007300650076000F00DA65006E00740067
S11307107300640000000000FFFFFFFF46534556CE
S1130720454E7E3120202012000000602C422C42D5
S1130730000000602C4202000000000042650072CC
S1130740005F0069006E000F00A864006500780077
S11307500000FFFFFFFF0000FFFFFFFF012E006D01
S1130760006500740061000F00A86400610074005B
S113077061005F006E000000650076004D45544145
S113078044417E3120202022000000602C422C4273
S1130790000000602C42000000000000412E0054C4
S11307A0007200610073000F00256800650073008B
S11307B00000FFFFFFFF0000FFFFFFFF5452415303
S11307C048457E3120202022000000602C422C422B
S11307D0000000602C42000000000000422000499C
S11307E0006E0066006F000F007272006D00610001
S11307F0740069006F0000006E000000015300796E
S1130800007300740065000F00726D002000560034
S11308106F006C00750000006D006500535953545F
S1130820454D7E3120202016000000602C422C42D1
S1130830000000602C42030000000000494E464FB7
S11308402020202054585420000000602C422C42C8
S1130850000000602C420500010000005354415484
S11308605553202054585420000000602C422C4240
S1130870000000602C420600010000002E20202011
S11308802020202020202032000000602C422C4216
S1130890000000602C420200000000002E2E2020E8
S11308A02020202020202010000000602C422C4218
S11308B0000000602C420000000000004E4F5F4C1E
S11308C04F47202020202020080000602C422C428A
S11308D0000000602C420000000000007B00330098
S11308E037003200300033004200460038002D004B
S11308F046004400380033002D0034003300320039
S113090031002D0041003400430034002D00390033
S113091041003900410042004600380046004200D0
S11309204300460044007D00000000002E202020EB
S11309302020202020202032000000602C422C4265
S1130940000000602C420300000000002E2E202036
S11309502020202020202010000000602C422C4267
S1130960000000602C4200000000000042470075B7
S1130970006900640000000F00FFFFFFFFFFFFFF9E
S1130980FFFFFFFFFFFF0000000000000149006EB1
S1130990006400650078000F00FF650072005600D7
S11309A06F006C00750000006D006500494E444501
S11309B058457E3120202020000000602C422C422B
S11309C0000000602C4204004D0000002B2D0000AC
S11309D02F2D0000412D00007F2D0000000000009D
S11309E0000000000100000001000000D10C000024
S11309F0880A0000980A0000A00A00000200000013
S1130A0000000000150D000034060000440600003C
S1130A10A00A00000400000001000000410D0000D5
S1130A20EC050000FC050000A00A0000080000001E
S1130A3000000000890D00001C0600002C060000C8
S1130A40A00A0000100000000000000000000000E8
S1130A50BC0A000000000000CC0A000000000000F6
S1130A600000000000000000000000000000000082
S1130A7000000000B1640000EF640000196600008B
S1130A80D1660000A0CAFF1F45670000C9670000C7
S1130A90E367000000000000000000001D68000083
S1130AA0A9680000AF68000017690000B56900007C
S1130AB0AD680000C169000089680000CD7A0000BB
S1130AC0CB7B0000BB7C0000F17C0000277D000094
S1130AD04B7D0000D37D0000677E0000777E000020
S1130AE07B7E00000000000038B504463D4D002028
S1130AF0C5E90000C5E90200C5E90400286268628E
S1130B00394800F0A0F8C5E906012046BDE83440A4
S1130B100FF2550100F05FB900F06FB970B5314DB7
S1130B200C46296A072904BF696A88421AD100F071
S1130B3093F8C0EB0016D5E90001D5E9022310189B
S1130B40B6FBF0F00A2148434FF49661B0FBF1F094
S1130B50401D0A21B0FBF1F04FF496614843206038
S1130B60002070BD012070BD2DE9F843064600F059
S1130B705AF81C4F0446386AD7E904598846421C7F
S1130B80D7E90601651B68EB0909494502D82CBF62
S1130B90A8420122012A3A6206D0042A08D0052A72
S1130BA00ED0072A0FD018E0C7E900487E6214E08F
S1130BB0D7E90001201A68EB0101C7E900010CE044
S1130BC0C7E9024809E0D7E90201201A68EB0101EC
S1130BD0C7E90201304600F010F9C7E90448BDE84E
S1130BE0F183000020C9FF1F803801001E48002146
S1130BF001606FF07F421D494A6000228A6007222B
S1130C000A601B491B4A0968C900B1FBF2F101B92A
S1130C1001214160704715480168C908C900016095
S1130C2000218160704710490A68134800680B6806
S1130C30C0430002000A9A42F6D1002110EB026080
S1130C4051EB1221704708494968A1FB0001C00813
S1130C5040EA4170C9087047054800687047024877
S1130C600168491C016070478CCAFF1F10E000E056
S1130C7024C1FF1F40420F0018E000E009010028D2
S1130C8006D5694A00F00F00801800F8041C70476C
S1130C90664A8154704750F82130120423F47023BB
S1130CA002F470221A430FE050F82100C0F30060F0
S1130CB0704706E0120202F4706242F0200203E080
S1130CC000BF120202F4706240F821207047F8E776
S1130CD0012800D0704710B5554C19B102290ED027
S1130CE004D310BD00206060206010BD4FF48070FC
S1130CF060605048016821F00201016010BD0322C8
S1130D0001212046FFF7D5FF2046BDE8104003220D
S1130D100021CEE700B1704710B5474C11B102294C
S1130D2003D010BD2060606010BD02220121204666
S1130D30FFF7C0FF2046BDE8104002220021B9E7BA
S1130D40012800D0704710B53C4C11B1022906D0DF
S1130D5010BD002020616061A061E06110BD072228
S1130D6004212046FFF7ACFF072205212046FFF7A8
S1130D70A7FF072206212046FFF7A2FF2046BDE871
S1130D801040072207219BE700B1704710B52A4C99
S1130D9011B1022903D010BDE064A06410BD022289
S1130DA013212046FFF793FF2046BDE8104002229E
S1130DB012218CE780B501211D48FFF775FF48B16A
S1130DC01F484168080005D0012088471D494FF09D
S1130DD0FF30086001BD10B501280C460CD101217B
S1130DE03F20FFF74BFF18494FF0004008600A22EC
S1130DF000F016F81248446010BD012800D0704776
S1130E0080B512494FF00040086000213F20FFF7F1
S1130E1035FF002200F004F809490020486001BDB4
S1130E200121034837E7000018ED00E000E400E08A
S1130E3000D0044014F10F4000A0044000C004405E
S1130E4098CAFF1FA0D0044004E100E084E100E060
S1130E50C16E11F1010F01BF016F11F1010F416F5B
S1130E6011F1010F02D042F6A20101E042F6A30102
S1130E70C16270473EB504460D46684600F050F81E
S1130E8004F10C004019001B6168A268051DA94209
S1130E903CBF5318984208D2421A684600F046F8FC
S1130EA06068A1680818421B2946684600F03EF8AD
S1130EB002A9684600F066F802983EBD174838B5A6
S1130EC081680D69E96A012442F6A302914223D0A4
S1130ED005F1680100248A68DAB1496853428B42FB
S1130EE022BF40680368994221BF40685118491ED7
S1130EF088420ED34AF2C03105F16800FFF7BAFF09
S1130F00696F884206BF012442F6A00042F6A100A0
S1130F1001E042F6A400E862204632BD10C0FF1F83
S1130F204FF0FF310160002141607047F0B585B09A
S1130F3004460D461646684600F08CF801208DF8EC
S1130F400B00206801901B48009000208DF80A00D7
S1130F50ADF808007EB100F01BF9174F694638461A
S1130F6000F047F832462946384600F078F83868E9
S1130F70019000F013F901982060606830186060F7
S1130F8005B0F0BD38B504460D46207910F00300D5
S1130F9007D0694600220A60C0F104022046FFF728
S1130FA0C5FF206828600548016821F4802101609C
S1130FB031BD0000B71DC104002003403C80044043
S1130FC00B7A4A7A1B0703F0405343EA82728B7A06
S1130FD042EA8362CB7A1B0603F080731A43826071
S1130FE00B68436042F0007383604968016082606B
S1130FF07047E0B5164A136843F4802313600A7BF4
S1131000002A0A6800924A6801920DD14A7A02B114
S113101002228DF808200A7A002A14BF0222032231
S11310208DF809208A7A0AE000228DF808200A7ACD
S1131030002A14BF022203228DF8092000228DF811
S11310400A20C97A8DF80B106946FFF7B9FF07BD6E
S11310503C8004400FF24801102200F0BDB803E0C8
S113106011F8013B0370521E3AB111F00303F7D19A
S113107003E051F8043B0360121F042AF9D2002A4A
S113108003E011F8013B0370521EFAD17047016866
S11310908068C0F3017002282CBF080C88B2704726
S11310A021100000FFFF000000000000000000000D
S11310B070B53F4E04460D46D6E90001002908BF2D
S11310C0002805D14FF47A70FFF7BDFDC6E9000191
S11310D0657000202070C4E90200206170BD38B53D
S11310E004460D46607838B172B66078401E607070
S11310F00020207062B632BD9DB1207898B1FFF710
S113110092FDD4E90223801A294D9941D5E900239F
S113111000F092F82169814211D272B60020207049
S113112062B6022032BD15F1010F08D072B601205B
S1131130207062B6FFF777FDC4E902012561032040
S113114032BD4178FF2901D10120704772B6417840
S1131150491C417062B6002070470160704772B646
S11311600168491C016062B601680029FCD10120B4
S1131170704772B60168491E01E072B60021016031
S113118062B6704772B60B490020086062B67047B9
S113119072B608480168491C016070470548016837
S11311A0022900D2EAE70168491E01607047000085
S11311B0A0C9FF1F80CAFF1F62B38B0708D0521E4D
S11311C011F8013B00F8013B00F024808B07F6D1B5
S11311D0830740F0208000BF103A07D330B4B1E851
S11311E03810103AA0E83810F9D230BC530724BFA5
S11311F0B1E80810A0E8081044BF51F8043B40F8D7
S1131200043BD20724BF31F8022B20F8022B44BF41
S11312100B7803707047083A07D3B1E80810083A0E
S113122040F8043B40F804CBF7D25307E4E70268E4
S1131230531C0360117070471B4213D1094236D10D
S11312402AB18446B0FBF2F002FB10C2704700F0F2
S11312506BB8FCD30022002370470B00020000216E
S113126000207047904271EB030CF6D370B5B1FACD
S113127081F4B3FA83F52C1BA340C4F1200532FAA0
S113128005F63343A2405FF00046E64002E05B0807
S11312905FEA3202841A71EB030524BF2046294613
S11312A07641F4D302000B003000002170BD012A06
S11312B0CFD970B5140C20D0B1FA81F4B2FA82F50A
S11312C0C4F120046419B4F12006D6D3B2405FF00F
S11312D00044F440002502E052085FEA3303C61AD2
S11312E071EB020E24BF3046714664416D41F3D365
S11312F002000B002000290070BD0C46B1FBF2F186
S113130002FB11452D0445EA1045B5FBF2F402FB3E
S1131310145580B240EA0545B5FBF2F002FB1052C9
S113132040EA044070BD000070470000DFF830164A
S1131330C968C9680020086070472DE9F041DFF8EA
S1131340205682B0E86900248DF801404669002ED9
S113135062D0E968C9680A68012A4CD001F1080220
S113136074680023091DA04704001FBF42F21270D5
S1131370844242F2137084424ED1E868C168D1F8C5
S11313800880B8F1000F47D04E68377837B1132F73
S113139004DA806800EBC700083800E00020086227
S11313A000281CBF006800281CD02A69926969467D
S11313B005F120009047040016D19DF8000040B1CB
S11313C04FF4E750791EC840C00758BF42F2117469
S11313D00AD5EA68D268126A1268414630469047D4
S11313E0002406E042F210743946204600F040FA28
S11313F094B901200DE0086A48B14168080003D09F
S11314000DF10100884704460CB1002001E09DF86D
S11314100100E968C96808602046BDE8F68180B526
S11314200178002000F024FADFF83405C06941692E
S113143009698847022000F09BFABFF34F8FDFF859
S11314402405DFF82425016801F4E06111430160FB
S1131450BFF34F8F00BFFDE7DFF80405C068C06825
S113146014210C3000F0B6BA10B5044600F0ACFB01
S1131470FFE72178BDE81040FAE110B5DFF8E02479
S1131480126852690446A16860689047F1E710B594
S113149000F04AF8DFF8C804C068C06861680161F8
S11314A0082101770020217800F0E2F9BDE810401E
S11314B000F09FBD30B583B0DFF8A444A5680021D7
S11314C0019100916B4681684068AD6801AAC9B278
S11314D0C0B2A847E268D2680021116100998A0865
S11314E0019900F0D9F937BD10B5DFF8742492687A
S11314F0D26804466068A168C0B29047B9E710B5E5
S113150000F012F800F012F8042101770020B0E78F
S113151010B500F009F800F009F803210177002064
S1131520A168BDE81040CEE1044695E7DFF8300439
S1131530C068C068A168016161684161704738B5DD
S113154000F088F8002141610161007F042804D182
S113155028680069804704B90446E868C068017FC8
S1131560204600F085F942F21270844208D1E868FE
S1131570C068007F082804BFBDE8314000F078BD92
S113158031BD2DE9FC4100F065F8016921B9002065
S11315902070FFF7D4FF5AE00121217006694769E2
S11315A0002000900123E869D0F814C0DCF804C0DE
S11315B06A4601A9E0475FEA000805D0E869416985
S11315C0C9688847404603E0009830B942F2127077
S11315D0FFF7B5FF002020703AE0B04288BF3046E4
S11315E00090E868C068017F082913D10199C1609F
S11315F0009981610198009900F005FD804642F24E
S11316007D7080451CBF42F2747080450BD14FF051
S1131610000808E02B68019A00999B6838469847AF
S113162080460098C7190098361A06D0B8F1000F02
S113163009D0E8694169C96888474046FFF77FFFD8
S11316400020207003E0E868C0680661476100205C
S1131650BDE8F681C24D0446E868C06870472DE9CC
S1131660F047BF4D8AB00446E868C068016921B9F3
S113167000202070FFF763FF57E001212170066905
S11316804769C168027F212E2CBF4FF02008B04665
S1131690A9B1424601A8FFF78FFDE869D0F814C04C
S11316A0DCF808C00123424601A9E047A6EB08067E
S11316B006B1B0B3FFF743FF0020207035E0032AE2
S11316C008EB070907D12B685B6801AA4146384635
S11316D09847824614E0102A18BF4F46DDD190F88F
S11316E01DA0FFF755FD39462F69CDF800A04346EC
S11316F0FF6B01AA05F12000B8478246FFF74EFDB3
S1131700BAF1000F4F46C8D0E8694569AD680123B6
S1131710002201A9A8475046FFF711FF00202070BE
S113172004E0E868C0680661476100200AB0BDE8CB
S1131730F08710B58A4B1B68DB680446E268A16831
S11317406068984795E62DE9F0410546874C6E6838
S1131750D5F80880E868824920600027496810317C
S113176030B10A68904223BF4968491C814204276A
S1131770304600F0EEFC00B904272978384600F022
S113178077F89FB96660002000F0F2F82068C4F88A
S1131790088018B180F3088880F30988616840469E
S11317A08847BDE8F041002000F0E2B8BDE8F081D0
S11317B038B50446606800F0CCFC08B9042005E0A4
S11317C06568012000F0D4F8A068A847217819E0E2
S11317D0634A10B5044602F120001269D269211D42
S11317E0904746E638B55E4D0446FFF7D1FC00F05D
S11317F024F86D6B04F10C02A8470546FFF7CEFCF4
S113180021782846BDE8344032E030B583B0044640
S113181068460021002206C0514DFFF7B9FC00F0D4
S11318200CF8AD6B6A46A8470546FFF7B7FCA268FB
S11318306946284600F04BF837BD05F120002D69B4
S1131840A3686168704710B5FFF76EFE4448C1682D
S1131850C968A2680A6162684A6110220A77C0688E
S1131860C068E16841770020A168BDE810405BE0F2
S113187010B584B0A02201908DF80020002200F061
S11318806AF88DF80220029102228DF803200023C9
S11318904469A4680C225BE010B588B0A72300F06B
S11318A03AF80020531C8DF8033006E06C4651F8DA
S11318B0203004EB8004401CA3609042F6D300F077
S11318C021F800231AE010B584B0A3222FE010B54C
S11318D088B0AF2300F01FF802238DF8033040B91D
S11318E09008801C8DF80300029203A8FFF774FC93
S11318F001E000200290002300F004F86946A047AC
S113190008B010BD1648C0699DF803104469A46866
S113191089000A1D70478DF80030019000238DF86E
S113192001308DF80230704710B584B0B0228DF8C4
S113193000200190012200F00EF8029100228DF89F
S11319400220002302228DF803200C224469A4689B
S11319506946A0471FBD0248C0698DF80120704741
S113196010C0FF1F0CED00E00400FA05CCC9FF1FF6
S113197070B50446022C04D0002000F0B8FF012CFE
S11319800ED00026114D06E04019C16889680A008E
S113199018BF8847761C1820704341590029F3D199
S11319A074B9FFF7F5FBFFF736F901F04AF8084977
S11319B000200860012001F075F801F030F962B6EA
S11319C0BFF36F8FBFF34F8F70BD00BFE4090000FA
S11319D008ED00E0002201F08FB90000C449EFF3E4
S11319E01080486072B6704738B5C24D2B696C6878
S11319F0DB6A2246042105F1200098472B69DB6A43
S1131A006A46012105F120009847206800990818CA
S1131A10401E6060002032BDF8B5B64F0446786BB6
S1131A200D464042164600EA0401621AAA185242C0
S1131A301040424207F120003F697F6C6B46B84773
S1131A4048B99DF8000008B16C20F2BD3246294621
S1131A50204601F06CF9F2BD2DE9F04F89B09246B1
S1131A6080460C4603AA00F01CF906005BD1A708C7
S1131A70BF00E41B4FF0FF300690079005D02246CC
S1131A8007EB0A0106A8FFF797FBFFF7A7FF07EB91
S1131A900809984D4FB12E6976693B465246414636
S1131AA005F12000B047060009D144B12E697669DA
S1131AB0042306AA494605F12000B0470646DFF88C
S1131AC030B2DBF8040080F3108866BB9DF80C008C
S1131AD058B3FFF783FF87B104A80290414605A8D5
S1131AE00190534600F025F83A462E69D6F828802E
S1131AF005F12000C047060010D17CB104A8029073
S1131B0006AB05A80190082200F013F849462C6999
S1131B10D4F8288005F12000C0470646DBF804000D
S1131B2080F310880EB1304600E0002009B0BDE813
S1131B30F08FA8680069006DC0B20090704770B55E
S1131B40044688B00D4600204DF82020401C08288B
S1131B50FAD375B12026202D98BF2E466A46314609
S1131B602046FFF779FF002804BF3419AD1BF0D0DD
S1131B7000E0002008B070BDF8B504460D46FFF73C
S1131B802DFF5C4E5C4B37693F692A46214606F1BE
S1131B902000B847564F796881F3108898B9B16826
S1131BA00969096B79B1FFF719FFB0680069036D22
S1131BB021463469646ADBB22A4606F12000A04754
S1131BC0796881F31088F2BDF8B54A4CA1680969B7
S1131BD06668326801F1580589692B6800204F4214
S1131BE093421ED16968914225D1FFF7F7FE22691D
S1131BF0414992683E4D04F120009047696881F3A1
S1131C00108868B9A1680969096B39B1FFF7E6FE64
S1131C1000F03EF8696881F3108808B90121297041
S1131C20F2BD9A4207D217EA030104D01046FFF727
S1131C30A3FF0028F4D16968494239404A427168D7
S1131C408A42EDD2481C811A1046BDE8F44093E75D
S1131C5070B5154682B000222A700A46254C2669C2
S1131C60766C01466B4604F12000B04778B99DF8C4
S1131C70001029709DF8001049B11D4D297831B923
S1131C8000F006F808B16C2076BD0121297076BDFC
S1131C90A06800692269016D126AC9B204F12000CA
S1131CA0104770B50546134882B080680069006B20
S1131CB00E46144600B101202070FFF78FFE7042DB
S1131CC08008800041426A462846FFF7C1FF084960
S1131CD0496810B181F3108876BD81F310889DF8AE
S1131CE0000008B100202070002076BD0000000034
S1131CF068CAFF1F10C0FF1F6B66656B416882686E
S1131D008A4209D2891A416082660FF26121016018
S1131D10012181600020704742F2787070470FF211
S1131D20050113E0416ADFF8D4334A898282CA6824
S1131D30921E42604A689A4202D1097A022902DB61
S1131D4042F2757070470FF20D0100BF0160002070
S1131D507047000010B5044682B0606A416862684A
S1131D60A1610168C91E9142A16002D342F276705A
S1131D7016BD008910B142F2777016BD8DF80000CF
S1131D806946DFF87C2302F12000126992699047CA
S1131D909DF8000010B142F2817016BD2046FFF795
S1131DA0ADFF16BD38B5DFF858532B689B68044661
S1131DB0626A216EE06D9847A8B9A1682069491E3E
S1131DC0884203D328680069804760B900F03AF874
S1131DD000F033F80098616E884200D038E00FF2CA
S1131DE08D102060002032BD38B50446C44D00F08B
S1131DF029F82B68626AE06D9B6810219847D8B96E
S1131E00E06D1030E065206E10382066112828BF80
S1131E10BC480FD208B1BC480CE028680069804770
S1131E2050B900F00AF80098616E884200D00FE0C3
S1131E300FF239102060002032BD694604F11C0005
S1131E40FFF7A0B8616A102204F11C00FFF76EB816
S1131E5042F27A7032BD10B5044604F11C00FFF75B
S1131E605FF8206E11282CBFA648A748C8E0A44BF1
S1131E701B68426E016EC06DDB681847F8B50446F6
S1131E80B4F85A00C0F30321C0074CBF0825042549
S1131E90E66D042901D00420F2BDFFF779F904F1BD
S1131EA06002974F3C69646B2B46314607F1200072
S1131EB0A0470446FFF772F9002C14BF2046002007
S1131EC0F2BD70B5044642F27F76E56D284600F017
S1131ED040F980B1606E04F11801A8470646012E4E
S1131EE003D12046BDE8704008E7022E03D100F07C
S1131EF080F8002070BD304670BD10B500F15C0163
S1131F00031D1C684A685A60944202D242F27670F9
S1131F1010BD0A7AD20708D50A685C69A24204D1C6
S1131F20496811B19960002010BD90F85A10C90792
S1131F305CBFBDE81040FFF7E1BE42F27C7010BD0B
S1131F40B0F85A108A0707D4CA0707D5C1F303208B
S1131F50002808BFFFF738BE04207047684A12689B
S1131F6052695C30416800681047000070B504464F
S1131F7004F15805616A28461022FFF72DF95A2604
S1131F800120415D7618401C1028FAD32878F1B25C
S1131F90884202D042F2797070BD69780A2942F20F
S1131FA0127023D8DFE801F01A060A0E24121A165A
S1131FB0241C1E002046BDE870409EE72046BDE874
S1131FC0704048E72046BDE8704050E72046BDE831
S1131FD0704076E72046BDE87040B1E7002070BD50
S1131FE0042070BD2046BDE8704047E742F27B7094
S1131FF070BD10B5454C70212046FFF7EBFC4448FA
S11320002060002010BDF8B504460D4600200026CF
S1132010404FAE4217D03869C0F11000A91B09E047
S113202079B13B69325DDA55761C3A69521C3A61E2
S1132030401E491E0028F3D1386100F005F810B99C
S1132040E7E742F27D70F2BD3049324A4A6200202D
S1132050CA682AB10B69934209D0581C086101E08F
S11320608A6E12B9084609680847521E8A66704784
S1132070F8B5234C20680069804700283DD1234FE0
S113208097F85900042824D107F15C052E683046DE
S113209000F05FF8D0B10020FFF76AFC97F85A000F
S11320A0800711D5686868616168103160B10A6899
S11320B0904222BF4968491C814201D20420F2BDEA
S11320C080F3088880F30988A868B04742F27E70DC
S11320D0F2BD08280FD10220FFF74AFCBFF34F8F4F
S11320E00D480E4A016801F4E06111430160BFF339
S11320F04F8F00BFFDE742F27B70F2BD53544D5049
S113210010C0FF1FE91D0000A51D00005CCBFF1FD0
S11321101F1D0000D0CBFF1F0CED00E00400FA05EA
S113212038B504460D460020FFF722FC8048814A5A
S1132130056044604FF420411160016881F3088810
S113214081F3098840688047BDE832400020FFF7EA
S11321500FBC10B582B000281EBF10F1010F7649E4
S1132160884201D1002016BD6A46022100F08CFE8F
S1132170002418B90098007A00B10124204616BD45
S11321802DE9F04F6D4E6E4F85B0B0680069683030
S113219000903D460AE00099097C014205D0686937
S11321A0EA688169526828469047183528680028EB
S11321B0F1D10024A246CDE9024A4FF47A70FEF729
S11321C042FD05468B460821002000F0ADFE30B9E3
S11321D04FF42040D0F80480D0F8009001E0A046ED
S11321E0A14600F057FD002838D14046FFF7B1FF63
S11321F0A0B3FEF763FE88B3B068006990F8860068
S1132200C00703D449464046FFF78AFF0098408A36
S11322104FF6FF71884208BF41F28830A5FB0023C6
S11322200BFB0033CDE90223FEF7FDFC04468A468E
S1132230DDE90201002908BF00280FD0FEF7F3FCF6
S1132240DDE90223001B61EB0A01994206D301D8A0
S1132250904203D349464046FFF762FF3D4600E003
S1132260183528680028E3D00099097C0142F7D08A
S1132270E9680968284688470028F1D0002DD7D09E
S11322800AE00099097C014218BFBD4203D0F968F5
S1132290896838468847183738680028F1D12846B5
S11322A005B0BDE8F08F10B5FEF76CFF00F0A8FC98
S11322B0224C2169496804F120008847216921489A
S11322C0E06304F12000096C8847A0680068804737
S11322D0002000F0E7FBFEF789FC206800688047D7
S11322E0A06840688047FFF74BFFE061016919B1BE
S11322F009680A0018BF8847E069416919B109688B
S11323000A0018BF8847E0680068BDE8104000472D
S113231038B5FFF7C8FF094CE569E06840688047B5
S1132320E868C1680800F8D028468847F5E7000047
S1132330D8C9FF1F08ED00E01104000010C0FF1F02
S1132340E409000064C0FF1F7047000008B90420BE
S11323507047DFF8B4150968090E01F00F010F2961
S11323600FBF4FF480210FF2746232F8111089020A
S11323700022026041604FF48072012181604FF4B9
S11323800061C160DFF8841591F900309A40426120
S1132390C9788161002101610162416200207047B6
S11323A070B508B9042070BDC4690FF21061656886
S11323B00C222846FEF700FFDFF854650FF208618F
S11323C0681C30601422A5682846FEF7F5FE681CD8
S11323D0706002202060002070BD38B5040001D177
S11323E0042032BDDFF82C256FF03B4000F046F8A6
S11323F001D06B2032BD38E02DE9F04389B0164698
S113240080460D4600F0EAF9049B00F0E3F904006D
S11324101BD1009D019F7019461EB6FBF7F007FB08
S1132420106121B1401C7843461E00E07D19AE4284
S113243017D32802000ADFF8DC1440F010600860AB
S1132440DFF8D404814502D06B2420465BE000F021
S113245089F90446D8F81000010018BF8047002C01
S1132460E4D0404600F043FAEFE7204600F025FAB6
S11324700546204600F03BFA284632BD1060DFF8DE
S11324809804814270472DE9F04389B004465FEA1D
S113249002080F461D4608BF042034D000F09FF9FF
S11324A0039B2A463946204600F054FA5FEA0009A5
S11324B029D1009FDFF85C6402E00398C7192D1A44
S11324C0EDB158F8040B706039020398090A042826
S11324D008BF41F0C06006D0082805D158F8040BA5
S11324E0B06041F0E0603060204600F0E6F98146DB
S11324F02069010018BF8047B9F1000FDDD02046E4
S113250000F0F5F9484609B0BDE8F08370B5040061
S113251018BF002A01D1042070BDDFF8F803DFF8EA
S1132520FC63CDB246EA054505601029156845608F
S113253002D01139032903D2082B04BF51688160EA
S1132540204600F0BAF90546204600F0D0F92846A6
S113255070BD2DE9F04389B05FEA0008914614BFCD
S1132560B9F1000F04200E461D4647D000F037F99C
S11325700698401E064208BF05421AD1A919109CAC
S11325800020491E012C05D1002E04BF691E072915
S11325900AD10AE044B9FF2907D9B6F5000F03D3DD
S11325A0DFF87C23914200D3042038BBDFF8647346
S11325B00DE0652022E0796849F8041B0699082992
S11325C004BFB96849F8041B06998E196D1AADB198
S11325D03002000A40F0407038602006069940F04E
S11325E0FF1040F47F40042908BFB86002D00829D6
S11325F008BF786000F0B6F80028DCD083E7F8B5AF
S11326001546002818BF002D0C461E4601D1042093
S1132610F2BDDFF80073DFF80C23E1B242EA0141B6
S1132620396000F04AF958B979682960102C03D050
S1132630A4F11101032903D2082E04BFB96869600B
S1132640F2BD002818BF002901D104207047DFF82B
S1132650D802007800F00302022A08BF002005D047
S113266000F0C00080280CBF012002200870002068
S1132670704710B50A46002818BF002A01D104206B
S113268010BDDFF8A4321C78002104F00304022CEE
S11326901ED06FF03A41C3F8021054781178240424
S11326A044EA0161947841EA0421D4782143C3F8CF
S11326B0061054791179240444EA01619479D27999
S11326C041EA04211143C3F80A1000F0F6F8014668
S11326D0084610BD08B904207047DFF8502280E096
S11326E02DE9F04F89B0924680460C4600F076F80A
S11326F0059B52462146404600F02CF978BB6A46B9
S11327002146404600F03BF9009C029E6042714223
S113271008404542A54208BF75197E4F03E0AAEB65
S11327200B0A5C447519BAF1000F17D0281BD34665
S1132730824588BF83460598BBFBF0F02102090A55
S1132740000441F0807140EA0920396040F0FF0044
S1132750786000F007F80028E1D000E0002009B01C
S1132760BDE8F08F4046A8E02DE9F04389B08046EB
S11327705FEA03090D46164608BF042029D000F07D
S11327802EF8079B00F026F818BB009D109C614FA3
S113279005E007998A08761A09EB82094D19C6B132
S11327A02802000A40F000703860200640F0FF1054
S11327B040F47F407860D9F80000B860FFF7D2FF9A
S11327C00028E6D0119901B10D60129909B10022D7
S11327D00A6098E6324629464046BBE099466A4676
S11327E0CDE042EA01414B4A116066E02DE9F04137
S11327F080461E000D46174608BF042034D004232B
S113280000F0A8F880BBD8F814307A195F42C2F1FE
S1132810000C07EA0C0CCCF1000C2F40ACEB0707C2
S11328200021B7FBF3F7DFF808C10AE0DCF800E0A9
S1132830203C6FEA0E0E2EFA04F4E40748BF491C4C
S11328405D1995420AD2B5FBF3F4202C38BFDCF8AD
S113285004E0EED3D8F818E07445E7D319B1B942CF
S113286034BF022101213170BDE8F0810000000075
S1132870002818BF002A01D10420704709291AD85A
S1132880DFE801F00509090B0D0F11131517C068D6
S11328901060002070474068FAE78068F8E7006835
S11328A0F6E70120F4E74069F2E78069F0E7006A9F
S11328B0EEE7406AECE76A20704710B51D4C7021C2
S11328C0217000F03BF888B911490968204688470F
S11328D02078810601D5672010BDC10601D5682086
S11328E010BDC00701D5692010BD002010BD38B54A
S11328F00400200000F022F80500002D03D10E484A
S113290003494968884731BD4C800440280002408F
S113291078CAFF1F040002406B66656BFFFF00432B
S113292000048000FFFF004102000240FFFF00405E
S1132930180002400000024004F0014008B90420DD
S11329407047C06920B10068022801D10020704797
S11329506D20704708B9042070475B1E194208BFF8
S11329601A4201D0652070470368994221BF40682C
S1132970C0185118884234BF66200020704770B5D3
S113298005000E46144601D1042070BD20212046C6
S1132990FFF720F82868301A2060E8686060A968AA
S11329A06868B0FBF1F0A0600420E06008202061BA
S11329B060610420A061E061002070BD802101708D
S11329C002780A42FCD070470168F02212040A43DC
S11329D00260BFF36F8FBFF34F8F70470800100082
S11329E0180020003000400060008000C00000019A
S11329F080010002000300040006000080B51B49AA
S1132A001B4808601B491C48421A1C4888421CBFCA
S1132A10002AFEF7D1FB1A481A49091A18BF00F018
S1132A2099FA19481949091A18BF00F093FA184974
S1132A301848421A04D0BDE808401748FEF7BCBB4A
S1132A4001BD16484FF0FF31016041608160C160F3
S1132A50016141618161C16111480160416081602E
S1132A60C160016141618161C161704708ED00E0AD
S1132A70000000002C7F00007082000000C0FF1FD7
S1132A8020C9FF1F08D1FF1F00C4FF1F20C9FF1F5B
S1132A90488300004883000008D1FF1F80E100E064
S1132AA080E200E0F8B5504C504D0100207847D149
S1132AB0296861604E498968096901F16802137CDB
S1132AC0167F190901F0010106F0010681F0010CDD
S1132AD00CEA0606DB0803F0010787F0010C16EA8E
S1132AE00C0F444B08D02968090F4FF0A070491C03
S1132AF0B0FBF1F01860F1BD527FD24302F00F0237
S1132B00521C394302D00122022103E00221022A8D
S1132B1028BF1146561E3706491E07F07067090480
S1132B2047EA067601F47021314329603249B1FB4A
S1132B30F2F11960012100F00BF801202070F1BDC1
S1132B40012904D1002100F003F860682860F1BD78
S1132B50884281B046D00129284820D1022101733E
S1132B60002102E000BF0099491C00910099B1F5D1
S1132B70FA6FF7D3302101708179C906FCD4C1788A
S1132B8001F01F0141F02001C17000200090009865
S1132B90B0F57A5F26D200BF0098401CF6E709BB67
S1132BA0017841F0040101708179C906FCD5002146
S1132BB0017302E000BF0099491C00910099B1F52E
S1132BC0FA6FF7D304210170C17801F09F01C1703D
S1132BD0002002E000BF0098401C00900098B0F56F
S1132BE07A5FF7D301B0704760CAFF1F4480044086
S1132BF010C0FF1F24C1FF1F006CDC020040064010
S1132C0080B500F0ABF93148416B41F47851416330
S1132C10016821F4433141F44131016001BD2B4885
S1132C202B4A416B21F478514163016811400160E2
S1132C3070472648016B41F480210163016B49030D
S1132C4001D40020704723490A7842F080020A70B8
S1132C500A781206FCD4016841F4E02101601E48A0
S1132C60017841F080010170017941F002010171A4
S1132C700120704719481A4900680968C0F30360C5
S1132C80401CB1FBF0F0704701289ABF144800685B
S1132C90002070471348016841F4807101601249B3
S1132CA04A6822F480524A60026842F013020260C9
S1132CB000204FF4FA720B68C3F300331818521E45
S1132CC0F9D1FA288041C00F704700000480044005
S1132CD0FFF3F8FF0C2107404021074044800440E3
S1132CE024C1FF1F30B0044090F00F407047000033
S1132CF062F30F2262F31F4200B500BF1300964631
S1132D009446103928BFA0E80C50FAD85FEA417CF9
S1132D1028BF0CC048BF40F8042BC90728BF20F8BF
S1132D20022B48BF00F8012B00BD00F02FB9134659
S1132D3080B50A4601461846FEF73EFA002002BD59
S1132D4070B510F0030F0C46154612D0B0F1005FB9
S1132D500FD22118491EB1F1005F0AD3C0F1005609
S1132D6032462946FEF728FAA21B71194FF000508B
S1132D7001E022462946FEF71FFA002070BD10B577
S1132D8014460A462146BDE810400123FDF770BBF6
S1132D9070B50D0082B00446164601D1002076BD00
S1132DA06A4600F071F830B9009BDB685B68324614
S1132DB029462046984776BD70B50D0082B004467A
S1132DC0164601D1002076BD00F07FF800B14CE03A
S1132DD000F047F868B9009BDB689B6832462946D7
S1132DE0204698474E49002806BF009AD268002220
S1132DF00A6076BD38B504460D466A4600F044F8CC
S1132E00A0B90098C068406908B9662032BD294657
S1132E10204600F05AF810B142F2D87032BD009A40
S1132E20D268526929462046904732BD002DFCD114
S1132E30002032BD70B50D0082B00446164601D1A3
S1132E40002076BD00F041F800B10EE000F009F872
S1132E5030B9009BDB68DB68324629462046984738
S1132E6076BD6A46294620460EE042F2D87076BD09
S1132E7010B52B4C2168002029B109690A0002D041
S1132E8088470021216010BD70B542F2D873D2B1D9
S1132E90244C6468146011B915E01034146014688B
S1132EA08CB12568002D04BF6668002E01D1E66848
S1132EB04EB1A84224BF65688542EED30818401E6F
S1132EC0854228BF0023184670BD70B50918491EF5
S1132ED00022144B9C685D682469160104EBC2044B
S1132EE05834755966682468AC4208BFAE4205D0B0
S1132EF0864228BFA14201D3012070BD521C022A80
S1132F00E8D3002070BD10B50648446804E00068AA
S1132F10010018BF80471034E0680028F7D110BDC5
S1132F2088CAFF1F10C0FF1F10B582B000228DF8A1
S1132F3000200A46064C014604F120002469646C12
S1132F406B46A0479DF8000000B1012016BD0000AB
S1132F5010C0FF1F002200F059B800000948817812
S1132F6004290DD1017801F09F010170FF218278BD
S1132F70012A03D1044A1278520701D4491EF6D11A
S1132F807047000001E0074002D007401D48006878
S1132F90000B00F00F00C01E082830D8DFE800F056
S1132FA005080B0E1114172F1A004FF4804013E07C
S1132FB04FF4C04010E04FF400400DE04FF44040A7
S1132FC00AE04FF4803007E04FF4C03004E04FF4DF
S1132FD0003001E04FF480200321421E10420A4ACF
S1132FE018BF022152684B1CB0FBF3F0C0F1005330
S1132FF042F8103F6FF0604301FB00305060002046
S1133000704700BF0070044010C0FF1F401810F04C
S1133010030308D0C91A1FD3DB0748BF00F8012DEA
S113302028BF20F8022D130030B414461546103979
S113303028BF20E93C00FAD8490728BF20E90C0042
S113304048BF40F8042D890028BF20F8022D48BF4E
S113305000F8012D30BC7047C91818BF00F8012DC5
S1133060CB0728BF00F8012D7047000001280ED8B7
S11330700FF2240280560122012900F01F0102FAF6
S113308001F10CBF024A034A400942F8201070477C
S113309000E100E080E100E01A1B0000BFF34F8F65
S11330A00548064A016801F4E06111430160BFF379
S11330B04F8F00BFFDE700000CED00E00400FA05AF
S11330C0ECE7EBE7EAE7E9E701280ED80FF2240280
S11330D080560122012900F01F0102FA01F10CBF00
S11330E0024A034A400942F82010704700E100E018
S11330F080E100E01819000002280ED80FF2240223
S113310080560122012900F01F0102FA01F10CBFCF
S1133110024A034A400942F82010704700E100E0E7
S113312080E100E01F212300002101807047F0B5F9
S113313085B004460D4616466846FDF78BFF002011
S11331408DF80B002088019041F2210000900020AE
S11331508DF80A00ADF808008EB1FEF719F80E4F8D
S113316069463846FDF745FF324629463846FDF79D
S113317076FF3846FDF78BFF0190FEF70FF80198B4
S1133180208005B0F0BD008808800448016821F45F
S11331908021016070470000002003403C8004400F
S11331A040684A49405C704748498A6842B14A6865
S11331B013780370501C48608868401E886070470C
S11331C00021017070475A2807D1404A01238B54CB
S11331D00FF2090111615169084770473B49496978
S11331E008477FB5394D696104460FF2F8006168FC
S11331F050F82160684600F0ECF801208DF80800D2
S11332008DF8090002213248E86032482861A2683A
S1133210606890476946304600F08CF82E49304685
S113322000F009F960680121FFF720FF616849197E
S11332300120887004B0002070BD70B50546234C91
S113324068680119897889B10FF2980151F82060F2
S11332500021FFF70BFF304600F0C7F86868AA6842
S113326000219047696809190020887070BD1748CB
S11332704160826081680029FCD10020704770B5EC
S113328004460FF2600082B050F82450E86A00014E
S11332900BD54FF0006007E0F168684688479DF859
S11332A0000068634FF00070E862E86A074E80012E
S11332B0F2D4E86A800308D5A86B4FF40031E962C0
S11332C021463269C0B29047F3E773BD94C0FF1F33
S11332D0A9310000C73100000000020A0020CEE737
S11332E00120CCE700C0024000D00240010C01F1F3
S11332F0804101F58E2101230A6803FA00F010438E
S1133300086070470029016814BF21F4804141F42A
S113331080410160704700210FF2501252F82130B1
S1133320834202D0491C0229F8D308467047012180
S11333302046E7E738B504460D46FFF7ECFF00F0FA
S113334043F8FFF7F4FF00F088F8012220684000FA
S11333504008206020680840297B40EA8170A97BEE
S113336040EA8160697B40EA0160E97B00F019F87A
S11333700121204600F054F8287804EB8000C1684D
S11333806A6800F014F82A7A920602F08062114307
S11333906A7A520602F000721143C16000F00FF81D
S11333A031BD090201F44071084320607047521E88
S11333B0D20621F0FE4102F0F0421143704720682A
S11333C040084000206070470FF2A80151F8200027
S11333D08CE70021017008214160002101724172D3
S11333E0017341738173C173704710B504460021A2
S11333F0206800F034F8FFF79BFF00F02CF80FF280
S1133400740151F82000010C01F1804101F58E2175
S113341001230A6803FA00F022EA0000086010BDE4
S11334200368090401F47C11012A0CBF194323EA3F
S11334300101016070478A0103D5026B22F080729A
S113344002638A0303D5026B22F480320263026BA7
S113345011430163704720465DE72068024940F04C
S11334600100206070470000FFCCFFBA00C002409A
S113347000D002400C003C100D003C10012100F073
S11334801F029140DFF86425400942F8201070477C
S1133490016841F00071016001688901FCD4704742
S11334A0016821F080510160016821F080410160D0
S11334B00168C901FCD47047016841F08041016092
S11334C0016841F0805101600168C901FCD5704771
S11334D038B50D46032D044602D1FFF7EDFF05E094
S11334E0042D03D1206840F0004020602046FFF7FF
S11334F0E3FF25B9206820F4000020600BE0012DD3
S113350003D1606840F0080004E0022D03D1606834
S113351040F48050606022E038B50D46032D044627
S113352002D1FFF7BDFF05E0042D03D12068400060
S1133530400820602046FFF7BFFF25B9206840F40B
S1133540000020600BE0012D03D1606820F008002A
S113355004E0022D03D1606820F4805060602046AE
S1133560BDE832409CE74068DFF884144018807856
S113357070475A280BD1DFF87824891801238B70FF
S11335800FF20D01DFF86C34596551680847704734
S1133590DFF85C1449680847F0B504460FF2B04000
S11335A0DFF8506487B050F8245002A800F050FBB4
S11335B001208DF80C004FF6FF7C10208DF80D00D3
S11335C006F13807DFF830048068016901F19402DC
S11335D0138863451ABF5B055B0D40F22313BB825E
S11335E0528862451ABF5205520D40F22132FA82C6
S11335F091F8911001F00F020F2A02D10120B87442
S113360024E00022BA740A071BD505223A74006923
S1133610B0F89200020A8DF80020420902F0070275
S11336208DF80220820800F003008DF8010002F0FA
S11336300702080900F007008DF803208DF8040044
S113364006E001F007000528387401DB0420387413
S1133650DFF8A803F86197F9100018B1022807D021
S113366003D308E0DFF8980307E04FF47A3004E06E
S1133670DFF8900301E0DFF890030290002106F1E7
S11336800800FDF715FD002106F12000FDF710FDEF
S1133690082030600920706002A9DFF870232846F2
S11336A000F057FA29684900490829602968C902C5
S11336B0FCD4686840F48040686097F910000528DD
S11336C006D1042038746946284600F0CEFA07E093
S11336D00FF2603100EB80004118284600F0C5FA73
S11336E0B87C28B10120787401212846FFF7F0FE48
S11336F0002038700820786000208DF8180001231D
S1133700F88AC34901EA8040059005AA00208DF893
S113371019000821284600F0E4FAA86A40F48070F1
S1133720A86200220020387209210820F860284687
S113373000F0C3FA0FF220302056FFF79FFE0FF27D
S11337401C302056FFF79AFE0FF214302056FFF774
S113375095FE07B0F0BD38B5A54D044669606068B4
S1133760A268022190476068FFF716FF6168012094
S11337704855002032BD38B504469D4D6068415D12
S113378061B10FF2CC2151F8200000F041FA6068D9
S1133790A2680021904761680020485531BD2DE999
S11337A0F043DFF8508283B004468946154600266C
S11337B008F1440711E00820386008364FF47A70A5
S11337C00190CDF8009008F1400260683B8909211E
S11337D0C0B200F00DF838688144AE4205D2A81B8F
S11337E00928E8D238602E46E8E70020BDE8FE83C9
S11337F0F0B50C460FF2582185B051F820501078DE
S1133800009960F3555100915068009960F3134199
S1133810009101987E4900F0604001EA8341084329
S11338200190009820F4801000900A98D0B10021F3
S11338300291039107E0C1F10707039EFF00BB401B
S113384033430393491CC9B2536899420AD20B5CAF
S11338500429F0DAC1F10307029EFF00BB403343A1
S11338600293EFE76A46E1B2284600F05CFAA0B999
S1133870012000FA04F6A86A5E4F3043A8620B9C4C
S1133880214607F10800FDF72AFC0328F8D0A96AAD
S1133890B143A96210B1052000E0012005B0F0BDDC
S11338A00FF2AC1151F82000016A4FF60241016297
S11338B0704770B506460FF29810564D50F82640E2
S11338C0A87860B3206A697801291FD144F20801FD
S11338D0084209D010F40C4F06D101212046FFF70D
S11338E01BFE002068701AE02878401E40B20028B1
S11338F048BF0420287095F900100FF2381001EB2E
S113390081010918204600F0B0F908E010F44C4F8A
S113391005D02046FFF7BCFD3046FFF73DFE206A88
S11339204FF60240206270BD2DE9F04180460FF24F
S1133930201086B050F82850286BA96A08400090DF
S1133940009800284AD02B4E30680099C140C8071F
S113395039D506F12000FDF7F4FB316801AAC9B29C
S1133960284600F013FA70BB0027002406E09DF8F7
S11339701070726D414638469047641C0198E4B259
S1133980C0F3034084421EDA072CF2D8DFE804F0C7
S113399006090C0F12151805EBE7E8E79DF80F7000
S11339A0E7E79DF80E70E4E79DF80D70E1E79DF8F8
S11339B00C70DEE79DF81370DBE79DF81270D8E712
S11339C09DF81170D5E770680099C140C80744BFDD
S11339D006F10800FDF7B5FB00982863286A4FF646
S11339E00240286206B0BDE8F081000000E100E07A
S11339F070CAFF1F48C9FF1F10C0FF1F73350000A6
S1133A0048E8010020A1070040420F0000B4C404AC
S1133A100000FC1F90C9FF1F04E0002040E70020C5
S1133A2047E700BF00207FE700E000BF01207BE7FD
S1133A30FCE7FBE717030404040B03040404050375
S1133A400404040303040404020304040400000043
S1133A5000400240005002404D6000004C5F0000F6
S1133A604B5E00000029016806D049004908016046
S1133A700168C902FCD4704741F00041016001684B
S1133A80C902FCD5704700210FF2783252F8213078
S1133A90834202D0491C0229F8D3084670470168C2
S1133AA041F080410160016841F08051016001688A
S1133AB0C901FCD57047016821F08051016001689B
S1133AC021F0804101600168C901FCD4704702689B
S1133AD092000BD5406B000E00F00F004000C21D99
S1133AE0D2B28A428041C043C00F70470020704761
S1133AF0016821F4802101600168C902FCD40168D5
S1133B0041F00071016001688901FCD46FF040420A
S1133B10016841F4201141F00F01016080214160EE
S1133B204FF433014163002100EB8103491C102948
S1133B30C3F88028F8DB026142618261826400215B
S1133B40002200EB0113491C1029C3F88020F8DB84
S1133B5070477CB504460D461646FFF794FF00F007
S1133B6069F81043086000F062F82879002860685A
S1133B700CBF20F4005040F400506060012100F0BC
S1133B8057F82046FFF7B4FF20686979491EC00939
S1133B9001F07F0141EAC010A9790029616814BFCE
S1133BA041F4805121F480516160E979002914BF06
S1133BB040F4800020F48000297A002914BF40F4E6
S1133BC0803020F48030697A002914BF40F48020CA
S1133BD020F4802020600A212868484308BF01207F
S1133BE0B6FBF0F0401EFF2888BFFF208DF80000D0
S1133BF0694603208DF8020002208DF8030001209D
S1133C008DF804008DF80100204600F02EF873BDF5
S1133C1010B50446FFF76CFF00F009F82046FFF7E3
S1133C2032FF00F007F822EA0000086010BD00210E
S1133C30204617E70FF2D41151F82000010C01F1CE
S1133C40804101F58E2101230A6803FA00F07047D0
S1133C5000210171DFF8A8110160102141710021D8
S1133C608171C17101724172704738B500F022F858
S1133C7060684FF6F8710840606060686A78297877
S1133C80920502F4400242EA0161AA78D20402F4E5
S1133C9060121143EA78120402F4E02211432A79F3
S1133CA002F00702114308436060FFE72046BDE8C5
S1133CB0324000E704460D46F1E670B504460D4671
S1133CC01646FFF704FF04EB05108030002E14BFE6
S1133CD04FF0006100210160002141608160C160FA
S1133CE070BD2DE9F0410746884614461D46FFF78E
S1133CF0EEFE07EB0810002640F8806F46608660F1
S1133D00C66075B1216841602179012908BF4FF46B
S1133D1000166179012908BF46F4801646F08061D7
S1133D200160BDE8F081F8B506460F461446FFF77A
S1133D30CEFE06EB0710002550F8801F01F07061DD
S1133D40B1F1406F20D0016821F0706141F0006151
S1133D5001606168C900C90841602168C1F340522B
S1133D600AB14FF4C005C1F300520AB145F48015FD
S1133D7001F4702141F040610D43A1688160E16864
S1133D80C16005600020F2BD0120F2BD70B504469B
S1133D900E461546FFF79BFE04EB061050F8801FF5
S1133DA00A0E02F00F02022A18BF062A25D1436820
S1133DB06E68DB0006F0604656EAD3036B604E0D76
S1133DC02B6823F4001306F0010643EA46530E0D54
S1133DD023F4F81306F0010643EA065301F47021B4
S1133DE019432960022A8168A960C068E860A06854
S1133DF00CBF002041F2B94070BDA068012070BD25
S1133E0048E80100004002400050024004003C1019
S1133E1005003C10010C01F1804101F58E210123C4
S1133E200A6803FA00F0104308607047010C01F1BE
S1133E30804101F58E2101230A6803FA00F022EA89
S1133E4000000860704700210FF2382252F8213038
S1133E50834201D108467047491C0229F6D3002049
S1133E607047B0FBF3F04FF47A7330B5B0FBF3F066
S1133E70DFF80C32B3FBF0F3002000E02046441CD2
S1133E8003FB04F58D4238BF9442F7D320B90A22CC
S1133E905143994228BF012030BD01210170002106
S1133EA041708170C17001210171417100218171E2
S1133EB0C17101210172417281720021C1720173C9
S1133EC0016141618161C16170472DE9F04106469C
S1133ED00C469046FFF7B7FF00F057F806F58876D2
S1133EE0022030600123002030600F22A178607826
S1133EF0490441EA40003063E078E17A000400F4C8
S1133F00E02040EA0130217B40EAC120A17940EA67
S1133F100120E17940EAC100217A40EA8100617A16
S1133F2040EA4100A17A0843706140462169FFF7E5
S1133F3098FF0746616900F024F80546A16901234A
S1133F403F224046FFF78DFF39062A0401F07061D5
S1133F5002F470220002114300F47C5040EA01078D
S1133F60E16900F00EF800F00F003843B0616179A8
S1133F702079090141EA4010217808433060BDE806
S1133F80F08101230F2240466BE70FF2001151F834
S1133F9020003FE780B50221C0F810110021C0F8CD
S1133FA01011FFF750FF0FF2E40151F82000BDE8B3
S1133FB002403BE7002211F440610AD04B0548BFA0
S1133FC04FF4627203D40B0548BF40F28732C0F845
S1133FD01411104670472DE9F04700F042F8BFB1C4
S1133FE000F03BF820B1ACB1A9EB0701216011E06E
S1133FF040F201300642F3D0F00703D51AF8010B62
S1134000E8647F1E16F4407FE9D04FF440702860C6
S113401000F02FF8BDE8F0872DE9F04700F021F813
S1134020BFB100F01AF820B1ACB1A9EB07012160CF
S113403011E040F202300642F3D0B00703D5E86D38
S11340400AF8010B7F1E16F4407FE9D04FF440704C
S1134050286000F00EF8BDE8F0872E68314640462F
S1134060A8E7804691468A461C464F4608F58A755D
S1134070704714B1A9EB07002060002070470000CE
S113408040420F00006006400070064006003410F5
S11340900700341000210FF2641252F821308342D9
S11340A002D0491C0329F8D308467047F8B50D46D9
S11340B0044628680101B2FBF1F6B6B206B901263E
S11340C05301B3FBF1F1A1EB46175100720112FA4F
S11340D087F2B1FBF2F1091A6422B0FBF2F000EBB3
S11340E04000884202D240F2F530F2BD2046FFF78C
S11340F0D1FF00F04CF81043086007F01F01E0788E
S113410000F0F300E070207800F0E00040EA2620A0
S113411020706670A07A00F0E0000843A072A078D6
S1134120297900F0EC000843A070207869794901EE
S113413000F0DF0001F0200108432070A879E0744A
S1134140E8796075207C40F088002074607C40F041
S1134150C0006074E078297A09B140F00800697AF7
S113416009B140F00400E0700020F2BD80B5017D8B
S11341700029FCD101794906FCD50021C170FFF763
S113418089FF00F004F822EA0000086001BD0FF284
S1134190780151F82000010C01F1804101F58E21D4
S11341A001230A6803FA00F070474FF4E13101601B
S11341B000210171417181710121C17100210172DC
S11341C04172704702780A430270C27842EA1122AF
S11341D0C270827942EA11428271427C42EA1161E0
S11341E04174704705E003791B06FCD511F8013BC7
S11341F0C37113465A1E002BF5D1704700A0064028
S113420000B0064000C006400A0034100B00341011
S11342100C00341070B5424E01243068491E154616
S1134220082900F10C024CD8DFE801F00514234200
S11342304228424B4000696811F1010F18BF002960
S11342400ED0D168012912DB90F8461001290ED155
S113425018300AE0696811F1010F18BF002901D173
S1134260002070BD116114701430FCF782FF00242B
S113427027E024212030FDF7ADFB22E0A9780029B6
S113428004BFE978002904D12978012908BF5470B2
S113429017D06A6829462030FCF78EFF30686968B9
S11342A0C16104731430FCF764FF0AE0052408E0DC
S11342B000211430FCF751FF306800211830FCF75E
S11342C04CFF204670BD38B50C460020012C0DD1A2
S11342D0134D286880F8461000F1200280682423DA
S11342E0022100F0C8F9296881F8474032BD002056
S11342F051B90B48006880F8482000F1200280681A
S11343002423022100F0B7B9704705490860002052
S113431070470349086000200968886070470000FE
S113432084CAFF1F10B5134601200BB9032010BD2A
S113433000225A745A6832B11468220003D00A4623
S113434001211846A04710BD10B5134601200BB932
S1134350032010BD00229A745A6832B114682200F6
S113436003D00A4602211846A04710BD2DE9FF419B
S11343700446002561688968227B4B7901209342B9
S11343804ED3096800294BD001EBC2010839002241
S113439000E0521C0B789A4242DA4B680C2606FB6A
S11343A002331E78032EF4D194F80EC0002100E0ED
S11343B0491C1A7A914205DA5A680E01B75C6745BE
S11343C0F6D1B518D978617355B3A5604FF00008DC
S11343D0974E984F07E0039402AA2068694600F0BC
S11343E059FA08F101082979884519DA00208DF86D
S11343F00400A86810F828008DF80200C009A96814
S113440001EB880101284988ADF80010A96801EB87
S1134410880149788DF803100CBF02970296DAE7F9
S113442004B0BDE8F08138B504460120A16861B14B
S1134430002506E0886810F82510206800F047FA87
S11344406D1CA1680A799542F4DB32BD70B504464F
S11344501546012084B0002D14BF002C03200BD07E
S1134460491E052908D8DFE801F05A0308182E442C
S1134470002121736174A174B9E0616800291EBF31
S1134480217B2A788A42F7D011B12046FFF7CBFF6F
S1134490287820730020A07311E061680029EBD014
S11344A02988627B0D460904B2EB116F0AD1A17B06
S11344B0EDB28D4206D02046FFF7B5FFA573204626
S11344C0FFF754FF93E0616800291CBFA16800292D
S11344D0F8D00026A26811798E42F3DA926829781E
S11344E012F82620914204BF206800F008FA761CD6
S11344F0F0E7616800291CBFA168002977D0002675
S1134500A26811798E4272DA9268297812F826200C
S1134510914204BF206800F0FCF9761CF0E729689A
S11345200A7802F01F02012A02BF0A79637B9A42C9
S11345305DD14A78012A20460AD0022A13D0032AE0
S11345401AD0092A22D00A2A40D00B2A45D04DE09D
S11345504988090A8DF808106A46296849888DF83F
S11345600910032120E063681B6804F10F02042191
S1134570984704F10F0107E063681B6804F1100217
S11345800421984704F11001696030E04988090A60
S11345908DF80810296849888DF80910297B59B1CC
S11345A0A96801916A46092163681B6898470099C4
S11345B069600199A9601AE0696800916A46A9686E
S11345C00191062163681B68984710E04988090A2D
S11345D0E17329688A1C072104E04988217404F1E5
S11345E01002082163681B68984700E0052004B0A6
S11345F070BD70B50C461546002114230E4A03FB0A
S11346000126326822B1491C0129F7DB022070BD62
S1134610314600F01CFA50B9306808B9032070BD67
S1134620002030737460FF20B0732E60002070BDD2
S11346304943000025430000A4C6FF1F10B5040031
S113464001D1032010BDFFF7EEFE0021216061605F
S11346502173A17310BD10B5040001D1032010BD56
S1134660607C08B1022010BD206800F001F908B98F
S11346700121617410BD10B5040001D1032010BDE7
S1134680A07C08B1022010BD206800F0F6F808B93B
S11346900121A17410BD000010B5044600F0DCFA3D
S11346A00020206084F88D0000F0E0FA002010BDA6
S11346B038B508B9032032BD446844B100680D061A
S11346C002D5A468A04732BDE468A04732BD0620E5
S11346D032BD08B903207047436813B100685B69B1
S11346E01847062070473EB504460A7AD5090120CA
S11346F0102A02F00F0319D100220B212046FFF7E4
S1134700E8FF04F18C000221817000220021017075
S1134710002004EBC001401C1028CA600A61F8D3D1
S1134720A36801212046984700203EBD082B11D2E2
S113473045EA430204EBC203DA685AB10868009000
S113474048680190487A8DF8080069461A69DB6860
S1134750204698473EBD002918BF002801D10320F8
S113476070478268002A18BFFFF7BDBF0120704759
S11347702DE9F04107461400884608BF032053D0B2
S113478000F06AFA294D286805F18C0630B1717879
S11347908F4203D100F06AFA01273FE018B100F01C
S11347A065FA02273AE0777000F060FA0020C5F855
S11347B0088077703070002205EBC001401C10287F
S11347C0CA600A61F8D3012F19D80FF2F810686093
S11347D0174800281CBF174800280BD0164800288B
S11347E01CBF1648002805D0154800281CBF1548D2
S11347F0002809D12846FFF74FFF072014E0284678
S1134800FFF74AFF06200FE02A462946384600F003
S11348105AFC070004D0284600F019F8384603E093
S11348200220B07025600020BDE8F08114C6FF1F8F
S1134830C7500000355100006F510000DD510000E9
S113484083520000C55200000022002141E710B548
S1134850040001D1032010BD616821B120684968BA
S11348608847002060602046FFF716FF002010BD37
S113487001F00F0141F080011AE701F00F0117E781
S113488008B903207047426812B1006812691047E2
S11348900620704710B508B9032010BD002918BFC1
S11348A0002A12D08B7803F00F04082C0DD2640078
S11348B044EAD31300EBC3031468DC6052681A6142
S11348C00A46BDE81040022103E7042010BD73B579
S11348D0044601F00F05CE090CB9032076BD01AAE8
S11348E00321FFF7F6FE082D07D246EA450104EB43
S11348F0C1010022CA600A6176BD042076BD02B5FA
S113490001F00F01082902D26A4604210BE00420B9
S113491002BD02B501F00F01082902D26A46052141
S113492001E0042002BDFFF7D4FE02BD0000000038
S113493010B501230AB9042010BD891E062900F10F
S11349408C0417D8DFE801F004060E10080A1200E0
S11349500C210CE00D210AE0A07800E0207800236F
S1134960107007E0062102E0072100E00921FFF7AB
S1134970B0FE0346184610BD10B50123032900F10B
S11349808C0406D0062906D0072908D0092913D09B
S113499016E00E2111E09AB11078002307E0A17807
S11349A0032906D062B11078207000230320A07080
S11349B006E02246082100E00A21FFF78AFE0346AA
S11349C0184610BDC7500000355100006F5100005B
S11349D0DD51000083520000C552000010B50446AA
S11349E000F03AF900F027F851B1817C8C4207D1EC
S11349F0002101604160817400F038F9002010BD8D
S1134A0000F034F9042010BD38B500F017F800F0B8
S1134A1012F819B1817C8C4200D113E007E038B55B
S1134A2000F00CF800F007F88C4200D10AE000F026
S1134A301DF9042032BD61480168704704460D46E3
S1134A4000F00AB9286000F011F9002032BD38B531
S1134A50FFF7F4FFFFF7EFFF21B1807C844201D11F
S1134A602960F0E7E3E7F8B50C46154601261DB1C9
S1134A706946FFF7D4FF08B10420F2BD002705E022
S1134A80491CC9B2032907D37F1CFFB200984068B0
S1134A90017A8F421CDA002102680C2313FB0723DE
S1134AA00FF28412D3F808E09EF804E002EB011C34
S1134AB09CF80C207245E3D15868DCF808302A468B
S1134AC021469847052804D00028DDD10026DBE7DD
S1134AD03046F2BD70B582B00D46044616466946AE
S1134AE0FFF79DFF88B9012D08D10099204600F0F9
S1134AF06CFF009A02212046FFF7B5FF009B5B681C
S1134B005B68324629462046984776BD2DE9F8432E
S1134B10914601240F46B9F1000F18BF002F8046BB
S1134B2001D0786808B9042045E000F095F8234ED8
S1134B30306828B1B17C884502D100F097F816E0BE
S1134B4018B100F093F8022411E086F8128000F006
S1134B508DF8776032461A494046FFF709FE040093
S1134B6007D03068FFF773FE4046FFF737FF204653
S1134B7021E000270FF2B00415E0002570680068FA
S1134B800C2111FB07012B01886800791A19127B8B
S1134B90904203D11B590A1D404698476D1C032DB2
S1134BA0ECD37F1CFFB27068007A8742E5DB306883
S1134BB0C9F800000020BDE8F283000000C6FF1F12
S1134BC0D54A000070B582B004466946FFF71CFF61
S1134BD0050027D1002517E00026009840680068EA
S1134BE00C2111FB05000FF240018268127901EBE0
S1134BF006110B7B9A4202D1406849688847761CAB
S1134C00032EEAD36D1CEDB200984068007A854209
S1134C10E2DB00980068FFF71AFE050004BF204697
S1134C20FFF7DCFE284676BDF34500003D46000054
S1134C304D44000001000000597100004D72000055
S1134C406972000003000000000000000000000082
S1134C5000000000000000000A480178002900D18B
S1134C6072B60178491C017070470000054801784C
S1134C7000291FBF491E0170C9B2002900D162B6C4
S1134C80704700001CC9FF1F2DE9F04104461D4672
S1134C900E461746FFF7E0FF47EA460804EB081004
S1134CA006F00F02C16A41F48043C36207F00101B8
S1134CB06668760A760246EA42165B0A46EA0116F6
S1134CC003F0080333435D606368C06A5B0A5B02F8
S1134CD043EA421242EA0111420A02F00802114375
S1134CE0069A92054009920D00F0400040EA024005
S1134CF040F088000860FFF7B9FF00F00CF9BDE848
S1134D00F08180B5C16A4A0A02F0080212180C3216
S1134D10026221F400610022826241F400510822FF
S1134D204262C16200920022036A0021FFF7ACFFD5
S1134D3001BD70B5011DFF224B6883F888204B68C4
S1134D4093F8944044F0020483F8944000234C68A0
S1134D5084F898300E68760A03F00F04760246EA67
S1134D604416002500F038F846F0080600F034F840
S1134D7046F0100635600E68760A760246EA441458
S1134D8044F01804256000EB43150024EC62002570
S1134D905C0044F0010400EB0414E5624C6804EB8D
S1134DA083045B1C082B84F8C050D3D300F59070A7
S1134DB005704B6893F8944004F0FD0483F8944024
S1134DC04B6883F88C2089224B6883F884204570D3
S1134DD0486800F008F870BD35600E68760A7602FF
S1134DE046EA4416704790F8941001F0DF0180F809
S1134DF09410704770B50C888B78C97803F00F0253
S1134E00DB09012943EA420505D1B4F5806F0ED3CD
S1134E1040F2FF340BE0412C28BF4024816801EBB1
S1134E20820191F8C06046F0010681F8C06000EB91
S1134E300511002BCD6A25F48045CD6264F3090584
S1134E40CD62CC6A24F40064CC6224F48064CC6225
S1134E5014BF04210821846804EB820494F8C05030
S1134E60294384F8C01053EA020108BFFFF749FF41
S1134E70002070BD70B5044601F00F05C80940EA72
S1134E804506204600F0FDF9A06800EB85000021EE
S1134E9080F8C01004EB0610C16A890A8902C16255
S1134EA0002070BD70B5044601F00F00C90941EA45
S1134EB0400204EB0212D36A23F48063D36223F426
S1134EC00063D36200236668450145EA0115760A4A
S1134ED045EA462503F0010645EAC6052E6876072D
S1134EE005D5D66AB605B60946F008062E605B1CE1
S1134EF0022BE8D3A26802EB8002084392F8C03088
S1134F0003F0FD0382F8C03004BF2046FFF7F9FE2A
S1134F1000F001F870BDA06890F8941001F0DF0172
S1134F2080F89410002070472DE9F047044684B0BF
S1134F30A06808228030017C0270C1F30318606805
S1134F40400A4002C1F3C00A40EA4810C1F380019C
S1134F5040EA0A1040EAC1000068C0F30949C0F3FE
S1134F6083000D284AEA480004EB00150CBF012712
S1134F700027E86AC0F3803000284FD004F5907011
S1134F8007B1C170BAF1000F35D0A96A4944A962CA
S1134F906A6A561AE96A81F40061E96281F480510F
S1134FA0E96203D08905B9EB915F1CD2A96A01912A
S1134FB0296A0091E96A21F48041E9628905B9EB23
S1134FC0915F08BFB8F1000F1BD1C078696A04EB88
S1134FD0C000408A814214D22068002300220021AC
S1134FE0FFF746FC1AE02A6A334648F0800120465F
S1134FF000F0BDF812E059EA080111D10020019037
S1135000009048EACA108DF808008DF809706946C6
S11350102068FFF7A0FBA068FFF7E5FEBDE8FF8767
S1135020E96AC1F34033BBB963685B0A5B02490AAE
S113503043EA481201F00801114349682A6AAB6A3D
S11350409A18914206D0002302E05E5C9E545B1CD9
S11350504B45FAD300210170A86A4844A862696AE2
S11350600E1AB8F1000F0DD167B18021204600F06F
S113507008F9E06A40F40060E062E06B40F400602C
S1135080E06303E0E86A80F40060E862E86A80F4C0
S11350908050E862696A002918BF002E03D0800599
S11350A0B9EB905F08D2A86A0190286A0090E86A78
S11350B020F48040E862A4E72A6A33464146204649
S11350C000F08CF8AAE770B515460FF2CC3282B026
S11350D0136800930C4630BB144E86F8220106F583
S11350E092710098F161B060FF2180F88010002275
S11350F00121304600F0E6F80D48B1687060000AFE
S113510081F89C00B1687068000C81F8B000B16847
S11351107068000E81F8B4003046FFF70AFE2E6076
S11351203460002076BD062076BD0000B8C6FF1F9F
S113513000C4FF1F08B9032070478268FF2182F86A
S11351408010816891F88420002281F88420002155
S1135150826882F89810826882F89410806890F8C7
S1135160001141F0C00180F80011002070472DE9C2
S1135170F041804601F00F00400040F0010008EBD0
S1135180001782B0F86A1D460126C0F3803030B99A
S1135190B8623A627D62F86A40F40050F86201F045
S11351A00F04F86A8005800DA84238BF054698F8B8
S11351B0210148B90095386AB96A0B1801222146C1
S11351C04046FFF761FD0646B86A284302BF002C3B
S11351D04046FFF796FD3046BDE8F6812DE9F041E3
S11351E0044601F00F00400004EB001782B0F86A97
S11351F01E460125C0F3803010B9B8623A627E625F
S1135200F86A40F4005083059B0DF862B34238BF3E
S11352101E46BB6AD4F81CC09B18BCF1000F04F5F1
S1135220907211D092F800C0BCF1000F0CD1412E45
S11352300AD216F0030F08BF13F0030C04D020F4B5
S11352400050F862E369157001F00F08507830B926
S11352500096002241462046FFF716FD0546002E23
S113526008BFB8F1000F09D1F86A80F48050F862E1
S113527020F48040F8622046FFF743FD2846BDE84D
S1135280F681E0B501F00F03CA0942EA430200EBDC
S11352900212D36AC3F380338BB14FF0FF3301930F
S11352A0136A8DF80810009300218DF80910D16A53
S11352B021F48041D16269460068FFF74CFA00206E
S11352C00EBD0000F8B504460B46114601200CB98A
S11352D00320F2BD0C2BFCD8DFE803F007203036A6
S11352E03D676D70819D9D879A00A168002081F8BB
S11352F00001A068017F490703D5017F41F08001C7
S11353000177A06890F8081141F0100180F80811A5
S1135310A06890F8941041F0010143E0A068017F77
S1135320490703D5017F01F07F010177A06890F858
S1135330081101F0EF0180F8081167E000296AD034
S11353402046BDE8F44055E5002964D02046BDE878
S1135350F44009788EE500295DD00A78114620468C
S113536002F00F05D609FFF78CFF46EA450704EB68
S11353700710C16A41F48061C1624A0A6068400A48
S1135380400240EA451040EA061002F0080289058E
S11353901043890941F08C010160A06890F89410D1
S11353A001F0DF0180F8941030E0A1B32046BDE89D
S11353B0F440097876E571B3088027E059B30A7898
S11353C002F00F03082B26D2D00940EA430004EB75
S11353D00010C06A800A00F00100488016E0D1B1D4
S11353E00878A16881F8980010E0002545F0800154
S11353F0C9B22046FFF73EFDE9B22046FFF73AFD69
S11354006D1C082DF2D32046FFF793FC0020F2BD5B
S113541009B100200870F2BD00B970473EB50468B8
S1135420A06890F88050280744BF2046FFF77CFD11
S1135430E80712D5A168012084F8210181F88000D1
S113544069460020009010208DF80800002001908B
S11354508DF809002068FFF77EF9280615D5A168A4
S1135460802081F88000E06BC0F38020002802BF18
S1135470E06AC0F38020002807D080212046FFF78F
S113548011FD00212046FFF70DFDA06890F85C1186
S113549009B180F85C1137BD002007402DE9FC41BB
S11354A004460F46904620681E4601AA0621FFF7CF
S11354B03FFA9DF804000525012818BF00282ED1C5
S11354C038781F21084208D1206804F11002042111
S11354D0FFF72EFA0546207C18E000F01F01012991
S11354E002D10025258214E000F01F00022812D109
S11354F0B8888DF800006A460020ADF80200052146
S11355002068FFF715FA05469DF8020000F0030035
S113551020820220306004F11000C8F80000284600
S1135520BDE8F68170B582B0054600208DF8000014
S11355300C4628680DF101020621FFF7F9F99DF8E0
S113554001000526012818BF002801D0052076BDDA
S11355506078032804BF01208DF8000020781F2103
S1135560084208D1608801282BD128686A46102196
S1135570FFF7B0FA24E000F01F00022804BF60889F
S113558000281ED1A0880F2108420ED100F00F017F
S11355909DF8002041EAD0112868002AC9B202D03F
S11355A0FFF7ADF901E0FFF7B4F99DF800102868A2
S11355B0002919BF221D0521221D0621FFF753FAD8
S11355C00646304676BD38B500F0B6F89DF80000C2
S11355D003280BD0012818BF022801D0052032BDB2
S11355E068888DF800006A4607210AE020680022D6
S11355F00721FFF7C1F938B901208DF800006A4688
S113560006212068FFF7B8F932BD2DE9FF470646A9
S1135610904630680C469A4603AA06216788FFF72D
S113562087F99DF80C003D0A01284FF0050903D0C5
S1135630010018BF02283AD1E0880190012D02D15F
S11356406A46092129E0022D04D18DF808706A46C2
S11356500A2122E0032D07D18DF80A706A46A0883A
S1135660ADF808000B2118E0212D05D1A0888DF894
S113567008006A460C2110E0222D05D1A0888DF87F
S113568008006A460D2108E0232D0AD18DF8087020
S11356906A46A0888DF809000E213068FFF71AFACF
S11356A081460098C8F800000198CAF800004846EE
S11356B004B0BDE8F08770B5044682B01546206892
S11356C01E466A460621FFF733F99DF800000128BB
S11356D018BF002801D0052076BD0120306004F1F8
S11356E0100204F11000286011212068FFF7F2F97C
S11356F076BD38B500F020F89DF80000012818BFE9
S1135700002801D0052032BD002000F00EF8688882
S113571010B9012000F009F82068AA1C0321FFF742
S1135720A2F92068AA1C07213AE08DF800006A4615
S113573020680621FFF720B904460D4620686A4612
S11357400621FFF7F5B8F8B500F043F89DF800001E
S113575008B10520F2BD0120386004F1100204F103
S1135760100030601221287920822068FFF7B2F9F6
S1135770F2BD38B5FFF7E0FF9DF8000008B1052041
S113578032BDA888A97841EA0020208204F11002E1
S113579020680421FFF767F9206804F1100208214A
S11357A0FFF798F932BDF8B500F013F89DF8000042
S11357B008B10520F2BDA888208204F110022068F7
S11357C00821FFF7B5F804F11001316002213960B6
S11357D0F2BD04460D46164620681F466A46062159
S11357E0FFF7A6B838B504460120052A0D460FD1A7
S11357F029786022114205D0090603D4E98809B149
S113580003B90020C1012046BDE83440FFF777B852
S11358100598E9880268914238BF016003680498DA
S1135820026800212046FFF723F858B929780906B1
S113583008D5204601B0BDE83040002300220021F5
S1135840FFF71BB832BD2DE9F0418AB004460020B1
S11358500D460390049005276868904610F1010FE7
S113586018BFB8F1000F10D002AA06212046FFF796
S11358705FF8287A0FF2B01C002808F1080649D016
S11358806868082801D1286808B9052076E04188AD
S1135890718060258188B180C188F18042787270FE
S11358A0037833702B420AD15CF8225028002DD0A3
S11358B004AB03AA31464046A847074626E0B9B1DF
S11358C0180615D4980602D500F072F803E05806BD
S11358D01CD500F060F80700079804900698039020
S11358E014D1F388039A00212046FEF7C6FF45E051
S11358F0980602D500F05CF803E0580606D500F0DF
S11359004AF80746079804900698039004A8019063
S113591000232AE09DF80800032808D174785CF875
S1135920244004AB03AA31464046A04724E06868FB
S113593000281CBFF08800281FD0307801061CD432
S1135940810606D500F01DF801212046FFF78BF8EB
S113595007E0400606D500F014F80F212046FFF7B3
S1135960B9F8074604A80190012303A800903A4619
S113597031462046FFF736FF074638460AB0BDE8F1
S1135980F08128680690059600208DF8200005AA6D
S113599068680790704700200690059601208DF8EE
S11359A0200005AAF08807900F212046FFF792B83F
S11359B000200690059601208DF8200005AAF088A5
S11359C0079001212046FFF74EB830B585B0044654
S11359D014480290039101208DF8040002AA0020CB
S11359E08DF80300694680208DF802004020ADF850
S11359F000002046FEF74EFF050010D100208DF870
S1135A00020002AA69462046FEF744FF050005D0BD
S1135A1080212046FEF75BFF284600E0002005B009
S1135A2030BD0000475800009D540000255500007B
S1135A30000000002555000000000000C7550000CC
S1135A400B56000000000000B7560000F35600009B
S1135A504757000073570000A7570000002000E0DC
S1135A6001202DE9F04104460FF2C8106D4D82B0BB
S1135A7050F8248008F58A763768780748BFF06BB9
S1135A80B8070AD50023012269464046FEF7C4FA46
S1135A909DF800002A6921469047F8070BD500209D
S1135AA08DF800006846E9688847002301226946AA
S1135AB04046FEF790FAB80544BF4FF400703060DA
S1135AC0BDE8F38140685749405C704755498A688E
S1135AD042B14A6813780370501C48608868401EBD
S1135AE0886070470021017070475A2807D14D4AD9
S1135AF001238B540FF20901116151690847704762
S1135B004849496908472DE9F041464D88B00446A3
S1135B1069610FF22018606858F820604248806874
S1135B20006990F87970FF2F08BF10276846FEF7C8
S1135B30B4F98DF801706068A26802219047FDF7FE
S1135B4099F8024669463046FEF7BFF9D6F81001C7
S1135B5040F00100C6F8100140F20721D6F8180100
S1135B600843C6F8180106F59276306840F4806060
S1135B703060FDF77FF84FF47A72616858F82110AD
S1135B80B0FBF2F0294AB2FBF0F0002200E01A4622
S1135B90531C00FB03F7322FF9D322B9B0F5FA7F77
S1135BA004D8012202E0102A28BF0F22130612048F
S1135BB0D1F8280103F0706302F470221A431043F1
S1135BC0C1F828010121706840F481707060606838
S1135BD0FDF77AFA1648286101206168491988702E
S1135BE0002008B0BDE8F08138B505460D4C686862
S1135BF00119897869B10FF23C0151F82000FEF7D0
S1135C00C9F96868AA6800219047696809190020E1
S1135C10887031BD03484160826081680029FCD1ED
S1135C2000207047ACC0FF1F10C0FF1F40420F0090
S1135C30EB5A0000006006400070064010B50B46A9
S1135C40DFF8B444114601205B1E2268062B2ED8CF
S1135C50DFE803F0040A1519222D2C0039B3086873
S1135C60400A00F0CAF804E009B30868400A00F0EA
S1135C708AF8E0B12268012182F8591410BDB1B14B
S1135C8058328A6010BD91B102F158008860BDE8B5
S1135C9010400868400AB0E04FF400400860012258
S1135CA04FF4007048600A748860C860002010BD1A
S1135CB00020704770B5DFF840442060583000F091
S1135CC070F9256805F1580000F016FB06464FF4FC
S1135CD0846105F15400FBF77DFE20680021C0F8C3
S1135CE060644165002070BDDFF80C14086000207A
S1135CF009680865704738B5DFF8FC43206890F8F8
S1135D005C0430B9FCF775F92068012180F85C1453
S1135D104165206890F85D04A0B32168022081F8F1
S1135D205C0400F0CBF80500F7D0206800F25C407A
S1135D30C168002904BF0178022903D1032000F0BF
S1135D40E6F801E00121417042F27D70854219D0EC
S1135D50206800F25D400021017042F274718D42AE
S1135D6002D10221C17431BD42F212718D4203D1BC
S1135D700221C174032002E00321C1740020BDE8A4
S1135D803240C4E031BD70B50446B4F5847F82B0BE
S1135D900D4630D3D84E306800F25B410A7862B9C0
S1135DA0887808B10F2076BDA868694600F074F8B9
S1135DB008B3009800F097F803E0D0F86404844234
S1135DC019D130686A6800F264414B68934238BF65
S1135DD01A468E6896199B1A641C8E604B600C6080
S1135DE013B9002180F85B1400F51670A968FBF75D
S1135DF0E3F9FFF780FF002076BD38B50C46054671
S1135E006168A068FDF7A6F80FF2984000E00C3036
S1135E10416831B10268AA42F9D18268A068FBF7EF
S1135E20CBF90FF2043045B140F201116D1A0DD0D7
S1135E306D1F19D06D1E1BD027E0A168552081F875
S1135E40FE01AA20A16881F8FF011EE0A16801F506
S1135E50BE7400F01CF80A682260097C50F8210026
S1135E6000F04AFA206210E0A06800F09AF80CE012
S1135E7000F00DF8097C50F82150284600F03CFA57
S1135E800246A0682946FBF797F9002032BD9A49DB
S1135E90096801F58C6170474269984B9A4202BFC8
S1135EA0426B974B9A4204BF027E012A04D1C06917
S1135EB00001086001207047002070478E48006888
S1135EC0D0F86C24B2F5007F04D2110004D142F260
S1135ED07D7070474FF40071521AC0F86C2400F5BD
S1135EE01670FCF790B88449096801F25A420123FC
S1135EF01370537001F58D61002393700123D370E7
S1135F000023137108604B600120087270477A49BE
S1135F10096801F25A42012313709070002301F5BD
S1135F208D605370D370137101214360036001725B
S1135F30704730B53022027078224270002282729B
S1135F400FF2D0139400C4F11C0421FA04F505F0F7
S1135F500F041518E45CAC70521C082AF2D330BD4F
S1135F6010B5002261B10A23B1FBF3F30A2404FB48
S1135F70131130311154521C19460029F3D102E097
S1135F80302101700122002111541118491E05E02D
S1135F900A78037801F8013900F8012B8842F7D315
S1135FA010BD70B504465748C0B0806805692868BC
S1135FB014904FF6FF70B5F87A608642524808BFD5
S1135FC041F28836016826A8FFF7B3FF55F8101F81
S1135FD00DF1A300FFF7ADFF286869680818411E9A
S1135FE00DF1AE00FFF7A5FF69690DF1B900FFF7E8
S1135FF0A0FF6869A9690818411E31A8FFF799FF35
S1136000A96C0DF1CF00FFF794FFE96C0DF1DA00F4
S1136010FFF78FFF296D0DF1E500FFF78AFF696D2A
S11360203CA8FFF786FF696815A8FFF799FFA968E0
S11360300DF15F00FFF794FF29690DF16A00FFF786
S11360408FFFA9690DF17500FFF78AFF314620A87B
S1136050FFF786FF2D4801680DF18B00FFF780FFE5
S1136060AA6D2B4B22A023A19A420CBF0A460246DA
S11360702B6A03B108460F900DF18B033CA80E90D8
S113608013930DF1E5000D9020AB0DF1DA000C90A7
S113609012930DF1CF000B90119231A80A90109138
S11360A00DF1B90009900DF1750008900DF16A0029
S11360B007900DF15F0006900DF1AE0005900DF113
S11360C0A300049015A8039026A802909DF8500000
S11360D09DF852309DF853200FF25C0101909DF819
S11360E051000090204600F023F940B070BD00003C
S11360F06E6F00007965730094CAFF1F53544D50AE
S11361007367746C10C0FF1F2480044024C1FF1FF8
S11361106B63666730313233343536373839616210
S11361206364656600000000640600006C060000FD
S11361307C060000880600004B696E657469732054
S1136140426F6F746C6F6164657220256325642EE1
S113615025642E25640D0A0D0A53797374656D2028
S11361606465766963652049443A2025730D0A46BF
S11361706C6173682073697A653A202573206279AB
S11361807465730D0A466C6173682072616E67658D
S11361903A2025732D25730D0A466C6173682073AC
S11361A06563746F722073697A653A20257320627F
S11361B0797465730D0A466C61736820626C6F6351
S11361C06B733A2025730D0A52414D2073697A6529
S11361D03A2025732062797465730D0A52414D206B
S11361E072616E67653A2025732D25730D0A526519
S11361F073657276656420726567696F6E20303AE4
S11362002025732D25730D0A5265736572766564B6
S113621020726567696F6E20313A2025732D2573CE
S11362200D0A566572696679207772697465733AE6
S11362302025730D0A436865636B2072657365726C
S113624076656420726567696F6E733A2025730DF5
S11362500A426F6F7420636F6E666967207072659F
S113626073656E743A2025730D0A506572697068FF
S11362706572616C20646574656374696F6E207403
S1136280696D656F75743A202573206D730D0A432B
S1136290505520636C6F636B3A20257320487A0D48
S11362A00A00000000000000940600003600000010
S11362B001000000CC0600000E00000001010000F7
S11362C0DC060000A0010000030100007C080000BF
S11362D060000000040100002C090000A000000080
S11362E005010000DC0800004D0000000000000073
S11362F0000000000000000000F10103810704D049
S113630010F8011B89B18107FAD10268B2F1013199
S1136310914311F0803F04BF50F8042FF6E710F8C2
S1136320011B11B110F8011BFBE7C01A70470000F4
S11363300CB41CB5044604A801900A46009401ABB1
S1136340694607487844183000F018F8009A00218C
S1136350117000285CBF0098001B16BC5DF80CFB94
S1136360CFAEFFFF70B504461E000846154604D0A4
S113637015F8011BA047761EFAD170BD2DE9F04730
S113638084B08246894614461F46E84607E0012346
S1136390224649465046FFF7E5FF8146641C2078B3
S11363A010B904B0BDE8F0872528F0D16078A41CAA
S11363B02528014618D058285CD063280ED06428BC
S11363C018BF692814D06F2854D0702858D0732867
S11363D05DD0752818BF78284CD0E0E7386838605D
S11363E050F8041B3860C9B24846D0478146D6E706
S11363F03868386050F8045B3860002D03D52D21CF
S11364004846D047814664206F2808BF082205D03B
S113641040F02001782914BF0A2210220B2164289D
S1136420AC4603D1002D48BFCCF1000CBCFBF2F507
S113643002FB15CC0CF130065FFA86FC4B1EBCF156
S11364403A0FA4BFA0F15106B44403F808C019469A
S11364505FEA050C01D00129E8DA68460D184846C0
S1136460D1F10B09C2D015F8011BD047B9F10109CC
S1136470F9D1BBE73968396051F8045B3960C3E787
S11364803868386050F8045B38607820BCE73868B6
S1136490386050F8045B38602846FFF72DFF06008B
S11364A04846A3D015F8011BD047761EFAD19DE7C4
S11364B010B59B488068006900F1680434214AF2F1
S11364C0C030FCF731FD48B934224AF2C0312046CD
S11364D0FAF782FE20689349884204D0FF223421CF
S11364E02046FCF705FCFCF701FC002010BD38B584
S11364F08B4DA86804694B20E07004F1100202205F
S1136500A07004210020607020705020E0710120F0
S1136510A07102206071002020715420E0720120DB
S1136520A072002060722072012020634EF6FF707A
S1136530606305F120002B69DB6A98472B69DB6AED
S113654004F11402012100F063F82B69DB6A04F101
S11365501802002100F05CF82B69DB6A04F11C02CC
S1136560022100F055F82B69DB6A04F120020321B3
S113657000F04EF82B69DB6A04F14402052100F0B7
S113658047F82B69DB6A04F14802062100F040F861
S11365902B69DB6A04F14C02072100F039F8A06989
S11365A0614A404252424FF0FF310240891A5F4A29
S11365B0E1651040A06500215D4820665D48606685
S11365C06869E16007E094F87830134202D0E36828
S11365D01A43E260491C182202FB01021268002AD5
S11365E0F1D15548016821644168E1638068A06382
S11365F0686850F8101F616241680068081A401CFE
S1136600A0622046FAF724FC01202065002032BD58
S113661005F1200018470000F8B51446404A474FDA
S113662091680426401E096917281D464DD8DFE8E5
S113663000F00C121416181A20224C24262D4C1C7F
S11366401E30333F424446484C4A05B12E6004B1E3
S113665021600020F2BD0C31F7E71031F5E7143169
S1136660F3E71831F1E72031EFE72431EDE7283182
S1136670EBE73431E9E72C31E7E73031E5E7D0697E
S113668041694969884738603946DEE71026583140
S1136690DBE72B480068F6E702F1200012699269F3
S11366A0694690479DF800000028ECD00120EAE7F5
S11366B00C263831C9E74431C7E74831C5E74C31C6
S11366C0C3E75031C1E70831BFE742F63C00F2BDF1
S11366D0134A92681369401E072842F63E0218D9ED
S11366E009380AD0401E012884BFC01E032810D9CF
S11366F0083808D0801E0CD00EE0002918BF0129EC
S113670003D119637047032901D3104670471965F3
S1136710704742F63D00704742F63C007047000067
S113672010C0FF1F6B636667488300000000000011
S113673000C0FF1F07E1FF1F5880044058CBFF1F14
S11367402480044030B5044685B060686946FAF791
S1136750E5F9002835D16068012804D002280CBF6F
S1136760424D434D00E0434D01A8FDF71EFD009846
S1136770019001208DF80C008DF80D006068FCF785
S113678083FA024601A92846FDF790FCB0B9606877
S11367900121FCF7B1FC4FF400512846FDF712FD2E
S11367A06068A268344C0221904761685A20884787
S11367B06168A62088470120207003E06068FAF72A
S11367C093F9002005B030BD10B504462A48416055
S11367D06068A268012190476068FAF785F9002093
S11367E010BD10B504462448007870B160680021DB
S11367F0FCF782FC6068012804D002280CBF1B4807
S11368001B4800E01B48FDF7B1FC6068FAF784F907
S11368106068A268BDE810400021104780B5406858
S1136820012804D002280CBF1048114800E0114888
S1136830FDF7D8FC002002BD10480178890600D578
S11368400AE070470E4801788A0701D5C07870477E
S1136850890600D500E07047C078074949680847B1
S113686008480178890600D5F6E7704700C006405D
S113687000A0064000B00640E4CBFF1F04A0064081
S113688004B0064004C00640AF49D1F88820531C28
S11368905218C1F8883082F82000D1F8880000F03E
S11368A03F00C1F88800704700207047B8E02DE928
S11368B0FC410C00154614BF002D0420984628D036
S11368C0A14F002007F190062860707000F0A8F82E
S11368D018B11EE0A22000F075F820213846FBF71D
S11368E079F842463946684600F0F8F810B10021BC
S11368F029600EE03946684600F042F9BDF80410FC
S11369008142E7D1012030702760BDF80200286081
S11369100020BDE8F6812DE9F0410C0082B0154657
S11369201E4635D0212D33D200F07AF800283FD10D
S1136930DFF8148298F8910010B1002088F89100D3
S113694008F160075A203870A42078700EB1A52091
S113695078707D802DB12A46214608F16600FAF749
S11369602BFC08F16601384600F00AF9B880A91D2D
S1136970384600F064F8D8B9684600F0EFF8B8B9C2
S11369809DF80100A12812D0A22806D0A32801D086
S113699004200DE042F212700AE07888811D384626
S11369A000F04DF820B99DF80100A228E4D00020A1
S11369B0BDE8F681654801218170002101707047AE
S11369C02020704780B55A218DF800108DF8010001
S11369D001205D4981F891000221684600F02FF8FA
S11369E002BD10B50446594882B0017842788078D7
S11369F01140014211D10FF2B8100088ADF8000027
S1136A00022223695B6869462046984723690FF28E
S1136A10A4115B6808222046984742F2137016BD01
S1136A204A48017819B100210170A12004E081785D
S1136A3019B100218170A320C4E700207047444AA3
S1136A40D3690A46014618461B695B6818472DE955
S1136A50F14F8B461646FAF7E6F804464FF47A707F
S1136A6088467043FAF7EFF8DFF8DCA00027064603
S1136A7089460AF188050EE06868296888420CD0C6
S1136A805044009990F8200078547F1C6868401C9A
S1136A9000F03F0068605F451DD0FAF7C4F8021BA0
S1136AA061EB080341450AD828BFA04207D2E2435C
S1136AB06FEA080310185941421C41F10003B9F16F
S1136AC0000F08BF002ED7D04B45D5D301D8B24212
S1136AD0D2D3052000E00020BDE8F28F70B582B06B
S1136AE005460C46164600F039F858BB6878A628C7
S1136AF004D11748C069FFF774FF76BDA42106B11D
S1136B00A521884201D0012076BD00F023F8BDF80C
S1136B1000106980B0B908462128A8BF20206880E9
S1136B2000F018F8BDF80010A98058B9698849B177
S1136B302046FCF70FFA69880A2000FB01F2204680
S1136B40FFF785FF76BD0000ECCBFF1F7CCCFF1F59
S1136B5010C0FF1F14220221684678E710B50446CE
S1136B60002201212046FFF772FF40B920785A28FD
S1136B70F6D1601CBDE810400A22012167E710BD70
S1136B8030B583B004460D466846FCF7CDFA0422BE
S1136B9021466846FCF7CBFA628829466846FCF72A
S1136BA0C6FA01A96846FCF7EEFABDF804003EBD3A
S1136BB05AA70000000201500000AAEA05484CF25E
S1136BC02051C1814DF62811C1814FF4E971018032
S1136BD0704700000020054005207047087A18B966
S1136BE0184808604C2006E00520704705207047CF
S1136BF0154808601220486000207047087A18B9C8
S1136C00124808604020F6E70520704710B5887ADE
S1136C100F4A10B9136850680FE092680B89148901
S1136C20A34202D1042800DA01D1052010BD136863
S1136C30526853F8203052F8200048600B6000205E
S1136C4010BD000090C1FF1FDCC1FF1FF0C1FF1F7A
S1136C5034C3FF1F002101604160FB3041700170AB
S1136C600020704710B5044604F15800811C00222E
S1136C700A708A72CA7204F130010A6840F8142F4B
S1136C800A79D2094275C87998B303282CD004280C
S1136C903ED012281ED0152849D01A2842D01B28CD
S1136CA059D01D284DD01E282DD0232844D0252866
S1136CB033D0282813D02A2820D02F2846D055286E
S1136CC035D05A282ED09E2827D0A82807D0AA2805
S1136CD014D045E02046BDE8104000F03CBD2046FD
S1136CE0BDE8104000F049BD2046BDE8104000F06A
S1136CF027BD2046BDE8104000F08ABD2046BDE80F
S1136D00104000F04ABD2046BDE8104000F06ABEC5
S1136D102046BDE8104000F040BE2046BDE81040CB
S1136D2000F0C3BD2046BDE8104000F07EBD204603
S1136D30BDE8104000F093BD2046BDE8104000F0CF
S1136D40C9BD2046BDE8104000F072BE2046BDE833
S1136D50104000F05EBD2046BDE8104000F069BE62
S1136D60204600F08CFE04F1EC0100220A704A7007
S1136D70CA708A700A72CA7110BD2DE9F0410C46BE
S1136D8084B0154662682F1D12F1010F4FF00108FF
S1136D90284605F1ED0618D1317800291EBF39685F
S1136DA00968002965D095F83710282918BFA82943
S1136DB05FD1002101916A4621680291002100916E
S1136DC001213B681B68984753E0BB68934224BF8A
S1136DD09A1ABA60B279012A09D10020B07186F8F2
S1136DE001803070317B2868FDF789FD41E03278FD
S1136DF0002A02BF62680D2A2168327852B33968CA
S1136E000968002935D06168019121680291F96807
S1136E10009195F83710282918BFA82904D13B6898
S1136E201B686A4601219847B86848B1F8686168E8
S1136E300818F860284600F01AFB8046B868C0B904
S1136E40002030700D23317B286805F14802FDF7DE
S1136E500FFD0EE060680D2802BF0868DFF8D81344
S1136E60884206D186F80380717B00F0FAFA86F82E
S1136E7008804046D0E02DE9F0410C4684B09046AD
S1136E806268002612F1010F08F1340108F1EC07E1
S1136E90404608F1040515D17A78002A1EBF2A68F5
S1136EA01268002A0DD0C9782A2918BFAA2908D146
S1136EB001966A4621680096029102212B681B689C
S1136EC09847A8E0AB68934224BF9A1AAA603A7A1A
S1136ED0012A07D10120F8703E723E707E7200F0E4
S1136EE09EF898E03A780AB36268019222680292A6
S1136EF0EA6800922A6813681A0011D0C9782A290E
S1136F0018BFAA2902D16A4602219847A86850B13D
S1136F10E86861680818E860404600F0D7FA064659
S1136F20A868002877D1002038705EE038790028FE
S1136F3066D060681F2802BF686AC04A90425FD169
S1136F404A78F020024202BF8B78E024234257D1D2
S1136F50387B401C824253DA002B51D0112B4FDA7C
S1136F607E72AE60CE61B4484861A86A88613E71A1
S1136F70E86AE8620A78120602D410B1012000E03F
S1136F80002038700878000603D5E86A10B10120A3
S1136F9000E000207870787800281EBFB8780028B8
S1136FA0012039D14046FFF75DFE0646052E14D177
S1136FB03878012806D1F87808B901203872002001
S1136FC0387008E07878012805D1B87808B901202C
S1136FD0F871002078700220F8723878002804BF15
S1136FE07878002817D1F879A8B9797BD8F8000007
S1136FF00D2308F14802FDF73BFC0120B8720AE0BA
S113700000F00DF8797B00F00BF801203E71F87068
S1137010B870F8727871304604B0BDE8F081B97B7D
S1137020D8F80000FDF76BBC2DE9FF47044604F1D6
S1137030EC0660688068317C427900258A424FF012
S1137040010A22D3006800B300EBC1000838002114
S113705000E0491C0278914217DA42680C2303FBD2
S113706001221378082BF4D196F80FC0002000E019
S1137070401C117A884205DA516803015F5C674558
S1137080F6D15D18D07870740DB901204EE0A5607A
S11370904FF000096A4FDFF8AC8108E0039402AABC
S11370A020686946FDF7F6FB824609F10109287953
S11370B081451CDA00208DF80400A86810F8290026
S11370C08DF80200A96801EB89014988ADF8001028
S11370D0A96801EB890149788DF80310C1090129D8
S11370E007BF7073CDF80880B0730297D6E700200D
S11370F030707070F070B0703072F07101203071C7
S11371000020E0607071B071F072707A012803D1D0
S1137110B17B2068FDF7B4FBB17B20681F2304F129
S11371202802FDF7AAFB01207072504604B0BDE8A6
S1137130F08738B504460120A16861B1002506E056
S1137140886810F825102068FDF7C1FB6D1CA16844
S11371500A799542F4DB32BD2DE9F0413A4D86B00F
S11371600F462968144609B1022062E02946FDF75A
S11371706EFC060004D02846FFF76CFD304658E04C
S1137180286820B92846FFF765FD032051E06F60A9
S1137190002005F1F507F871FF206B68B8712E46E1
S11371A01B686A46052130469847804601980028A6
S11371B01CBF0099002938D09DF81010009AF9706E
S11371C06A61491EF970702202992962A8610399C3
S11371D069620021E96105F158010A700A22CA7145
S11371E000228A708A816A69521E02F47F431B025C
S11371F0150A43EA026305F47F452B43050A05F4A7
S11372007F4543EA126200F47F431B0243EA0063B2
S11372102B4343EA10600863C863CA6200208A6390
S1137220387078702660404603E02846FFF712FD68
S1137230012006B0BDE8F0815553425355534243F3
S1137240776E00007B6D00001CC8FF1F38B504007A
S113725001D1032032BDFFF76CFF05462046FFF73E
S1137260F9FC284632BD00002DE9F8430546160016
S113727014BF002D03204FF0010800F0EA802C1DFC
S1137280491E052905F1EE0706D8DFE801F0A80339
S113729006162D500020B873DAE0206800281EBFBF
S11372A0B87B31788142F7D010B12846FFF741FF0F
S11372B03078B8730020787311E020680028EBD090
S11372C03088F97B06460004B1EB106F0BD1787B54
S11372D0F6B2864207D02846FFF72BFF7E73284676
S11372E0FFF7A2FE8046B3E0206800281CBF606858
S11372F00028F8D04FF00009606801798945F2DA76
S113730000F0A9F810D1387828B92868FDF7F7FA01
S1137310804601203870787830B931782868FDF7D4
S1137320EEFA80460020387009F10109E4E720688C
S113733000281FBF60680028F8780128D3D04FF0D8
S1137340000917E000F087F812D13878012805D138
S11373502868FDF7DEFA8046002038707878012826
S113736006D131782868FDF7D4FA804600203870B9
S113737009F10109606801798945E3DB787A03281A
S113738018BF022813D13879012813D0387A01287C
S113739003D1F97A2868FDF773FAF97A28680D237E
S11373A005F14802FDF764FA0020387278723879E2
S11373B001284DD13878002804BF7878002847D1B7
S11373C03871387A012803D1F97A2868FDF758FA18
S11373D0397B00F046F800203872787238E0316862
S11373E0087800F01F02012A01BFFA7B8B88DCB207
S11373F094422DD14C78FE2C02D0FF2C11D027E0E2
S1137400934204BF4A88002A20D1C98802291DDA80
S113741000061BD505F1F80070603068C088B060C4
S113742016E0934204BF4A88002A0FD1C98869B97B
S113743000060BD42846FFF77CFE2846FFF7F4FD30
S113744080460020F8700120387101E04FF00508F3
S11374504046BDE8F2838068317810F82900814203
S1137460704728681F2305F12802FDF706BA3EB5C8
S113747000F061F8206AB0F1011F28BF4FF480309A
S113748001900199E068814238BF08460295019055
S1137490042163681B682046984700F046F804F10D
S11374A0ED0007D2017B019B029A2068FDF7E0F909
S11374B0054609E001214170857102218172057040
S11374C0017B2068FDF71BFA28463EBD3EB500F05F
S11374D032F8606AB0F1011F28BF4FF48030019088
S11374E00199E068814238BF084602950190032162
S11374F063681B682046984700F017F804F1EC0015
S113750007D2817B019B029A2068FDF7B6F90546F4
S113751009E00121C17005720221C1720570817BED
S11375202068FDF7ECF928463EBD6269A36921692C
S11375305A439142704704460025206900906A46E8
S1137540704710B5536884696343C36012688369E4
S11375505A430261012904BFBDE81040FFF787BF09
S1137560BDE81040B2E700002DE9F041044604F103
S11375706C050020296804F1580829B92165696857
S1137580002900D002219CE0687D0028686808F189
S1137590020704F1EF0640D020B9216500F0CAF8D3
S11375A078B961E0AA7D002A2ED088420DD200F07D
S11375B09CF802D100F093F801E000F0BBF8002839
S11375C052D000F086F8112053E0814209D100F036
S11375D092F802D100F083F801E000F0ABF860B952
S11375E06EE000F08EF804D100F098F800F079F81D
S11375F001E000F0A0F800285CD0012184F85410C8
S113760003213970112161E02165AA68B17A2068EB
S11376100023FDF72DF9022026E048B9F17A20680D
S1137620FDF76DF928682065012084F854000BE00B
S1137630AA7D5AB1F17A2068FDF761F928682065BE
S1137640022084F854000120307013E0884213D2E1
S113765000F04BF805D105F10C02002100F042F8CE
S113766001E000F055F810B984F8540002E000F08D
S113767030F8B87205202AE081420FD100F03BF8BF
S113768005D105F10C02002100F02CF801E000F016
S11376903FF8A8B1012184F8541015E000F031F846
S11376A005D100F03BF8002100F01CF801E000F0E7
S11376B030F848B998F82810012908BF022100D0F1
S11376C0002184F8541002E003213970B972BDE836
S11376D0F081012084F8540003203870704705F1CC
S11376E00C0201212046FFF72CBF081A206598F8E8
S11376F02800012870470020206598F828000128F8
S113770070470020206598F828002B6801287047EE
S11377106B68AA68F17A2068FDF7AFB8A069296898
S1137720B3FBF0F02861A26902FB1010206505F19B
S11377300C0270476B68AA68B17A2068FDF798B8A4
S113774000F1580101F11802122313605160012362
S113775000219374BCE038B500F1580101F14002F6
S113776000230FF23C341D5D9D545B1C242BFAD383
S113777001F118024031242368E070B500F029F8C3
S1137780282E04D159799B7943EA012102E0A82EDD
S113779000F032F8183201230EE070B500F019F849
S11377A02A2E04D159799B7943EA012102E0AA2EB9
S11377B000F022F81832002393742B6894604B4332
S11377C01360D1600023536001231374BDE870403B
S11377D0CAE600F1390300215D781C782D0445EADE
S11377E004649D7844EA0524DD782C4300F11805EF
S11377F000F15802EE7F704709D15E791979360499
S113780046EA01619E79DB7941EA06211943704712
S113781000E000BF00F15801002241F8182F0122B6
S11378208A7400224A600A749EE638B500F1580151
S113783001F1640200230FF28C241D5D9D545B1C36
S1137840082BFAD301F11802643108235160136044
S11378500021012311749374BDE8324084E638B5E5
S1137860044604F1580505F1640000210FF2542286
S11378708B5C0B54491C0829FAD305F11800082124
S113788001600121817405F16401416000210174EA
S11378902046FFF769FE94F83810C90704D5A91CDF
S11378A005220A7024228A7232BD90F8373000F122
S11378B05801252B01F1180203D1082313602C3140
S11378C002E00C23136034315160012191740021D2
S11378D0117449E62DE9F0410FF2C01186B0096830
S11378E0009100F1580890F83F5098F86C6000211E
S11378F00022002300F1140426B1A668002E14BF50
S11379000226032627680197D4F804E00397F400BD
S1137910F7000C37CDF808E08DF80340CDF810E0FF
S1137920BD4288BF3D466F46D2B201EB0804D75D25
S1137930521C491C042984F86D70F4D3002203AF4F
S1137940C9B2D75D01EB0804521C491C082A84F80B
S11379506D70F4D398F86C208AB100220CE001AF6A
S1137960DBB201EB0804DF5D84F86D705B1C491C1D
S1137970C9B20829F3D3521CD2B2B242F8DB0122B5
S113798008F118018A7408F16D024A600D60002242
S11379900A7406B0BDE8F041E6E538B5054605F1E0
S11379A0580404F1180000210160012181740021B0
S11379B0416001742846FFF7D7FD05F138010A7FBD
S11379C0022A0ED00A7802F01F02172A02D10022DE
S11379D00A7732BD01220A77A11C05220A702422EB
S11379E08A7232BD2DE9F041044604F13B0604F1EC
S11379F05805377805F118000021016000F038F8C7
S1137A008046707E022808D0F80706D501207076DB
S1137A100521A81C01702421817260680368180084
S1137A2003D000220721204698474046BDE8F08154
S1137A30F0E670B582B0044604F13B0504F1580049
S1137A40297801F003018DF80010002140F8181F77
S1137A5000F00EF80646687E022807D060680368C6
S1137A60180003D06A46082120469847304676BD60
S1137A7001218174002141600174204674E500F104
S1137A805801002240F8502F01220271052088700D
S1137A902020087300204873704700000000000095
S1137AA0008004022000000046534C2053454D49F9
S1137AB046534C204D4153532053544F5241474554
S1137AC0303030310000000000000000DFF8D8132F
S1137AD00A7B01F25A4100200B7803B10120DFF840
S1137AE0CC331A705870C97F002914BF104300208A
S1137AF07047000070B50024491E1546DFF8A8330E
S1137B00112903F1080603F279425CD8DFE801F099
S1137B10095B5B5B5B5B0B1A3D42474C51565B5BFD
S1137B20292E14704FE0002D4DD0012010702878BC
S1137B30507029783068FCF7C6FB2978B06CFEF7E2
S1137B40B7F840E0107800283DD02A88110A0229AD
S1137B5039DAC81880F87B24D2B23068FCF7C7FB46
S1137B6031E0002D2FD0507828702CE05DB32A88A6
S1137B70100A022807DAC01802F47F4190F87B0447
S1137B80084328801FE005241DE0E5B12946FFF7DE
S1137B902FF817E0BDB12946FFF730F812E095B190
S1137BA02946FFF733F80DE06DB12946FFF714F8C5
S1137BB008E045B12946FFF711F803E01DB1294655
S1137BC0FFF714F80446204670BDF8B50FF21030E4
S1137BD0B54C0078B64E8DF8000005464FF4906120
S1137BE02046F9F7F7FEFBF724F80028B06800698F
S1137BF00CD190F8781001F0EF0180F87810B0689B
S1137C000069C16821F01001C1602DE000F17C061B
S1137C104FF6FF71728830888A4208BF884209D0C3
S1137C20A44908723088000A487270888872708883
S1137C30000AC8727068A04F10F1010F04D010211F
S1137C40FBF772F900B977689C489D4E076004F50C
S1137C508F60002101800020A06020652060224602
S1137C603146FCF753FF08B10120F2BD30680069CA
S1137C7020652046FEF71EF830684068A060204664
S1137C80FCF743FB68B2010007D58E4A01F00F03ED
S1137C909A18402002F8040C02E08B4B4022C25494
S1137CA0012005F01F029040884A490942F821004A
S1137CB02068FCF7C9FD0020F2BD10B50020FCF7D8
S1137CC081FFA0B9784C2046FEF70EF82046FCF759
S1137CD020FB7F480168490309D57E4A4FF400110F
S1137CE011607D4A1160016821F48021016010BD9A
S1137CF038B56E4C794D0020207001206070F9F782
S1137D0047FAFDF7F8FFA878032803D10020A870EC
S1137D10FAF7AEF9F9F742FA287800B10120607059
S1137D200120207031BD10B55F4C002104F1140016
S1137D30F9F713FA002104F11800F9F70EFA04F127
S1137D401400F9F716FA002010BD2DE9F0410C00DB
S1137D50154614BF002D042039D00020286013B12B
S1137D60012B02D02CE0012600E002264F480078C7
S1137D7060B3DFF8348108F10807B87930B13868A6
S1137D80242308F120020221FCF775FC0120B871BC
S1137D904FF0FF3108F11400F9F7E1F9387EB042F1
S1137DA006D0012E08BF02280AD142F212700EE05A
S1137DB0B87EF97E40EA01207969091F814201D227
S1137DC0012004E008F12401216028600020BDE8BE
S1137DD0F0812DE9F0413548007800280C4615461D
S1137DE03ED0212D28BF04203BD213B1012B10D04B
S1137DF011E00327DFF8B080F9F7CAF908F10806A3
S1137E00707950B100207071F9F7C8F942F212701C
S1137E1027E00427EEE7012023E0F9F7BFF93776DE
S1137E2000207076B576280AF076002C18BF002D55
S1137E3005D02A46214608F12400F9F7BDF998F83F
S1137E40460001280CD13068242308F120020121C6
S1137E50FCF701FC4FF0FF3108F11800F9F77FF946
S1137E600020BDE8F08110B54469A4680023002215
S1137E700021A04710BD002070472020704710B596
S1137E80094C94F85C04022818BF032807D104F1B4
S1137E901400F9F772F904F11800F9F76EF9206883
S1137EA0BDE81040FDF7B8BA84CCFF1F04D1FF1F12
S1137EB010C0FF1FDCC1FF1F34C3FF1F80CCFF1F96
S1137EC088C0FF1F18ED00E000E400E000E100E0DE
S1137ED03480044084E100E084E200E0DED0FF1F4F
S1137EE03500000000F00BF8002801D000F00AF87B
S1137EF00020C046C046FAF70BFAFAF725FA01202B
S1137F007047000010B5074979441831064C7C4489
S1137F10163404E00A68081D511888470146A14236
S1137F20F8D110BD0C040000200400002D13000043
S1137F303B130000EC040000A8C9FF1F4C0600001E
S1137F40C4C0FF1F740A000000C0FF1F7C050000AE
S1137F50E409000000000000000000000000000030
S1137F60000000000000000000000000000000000D
S1137F7000000000000000000000000000000000FD
S1137F8000000000000000000000000000000000ED
S1137F9000000000E0C9FF1F20CAFF1F15420000B7
S1137FA0000000005CC1FF1F3D5C000000000000F9
S1137FB088C1FF1F70C0FF1FF57A00000200000097
S1137FC0000000000000000000000000A9310000D3
S1137FD0C7310000000000000000000000000000A5
S1137FE000000000CD5A0000EB5A00000000000021
S1137FF000000000FFFF0300010000000406000071
S113800000C0FF1FFFBF002001000000CC090000DA
S113801000000040FFFF074000000000D4050000FE
S113802000F00F40FFFF0F4000000000D4050000E7
S1138030000000E0FFFF0FE000000000D405000096
S1138040000000000000000000000000000000002C
S1138050000040018103400002034000830240000D
S113806004024000000000000200000028C1FF1FBD
S1138070000000000300000038C1FF1F01000000E1
S11380800100000048C1FF1F54C1FF1F010100008F
S1138090000000000200000030C1FF1F00000000CB
S11380A00806500164C1FF1F010000000100000028
S11380B074C1FF1F80C1FF1F030100000600FF09F8
S11380C001A101850119012901150026FF00750888
S11380D095239102850219012901150026FF0075D7
S11380E00895239102850319012901150026FF0033
S11380F0750895238102850419012901150026FFBD
S113810000750895238102C012010002000000409E
S1138110A2157300020001020301000009024000DD
S1138120020100C032090400000203000003092117
S113813000010001224C00070581034000010705EE
S11381400203400001090401000208065003070568
S113815083024000000705040240000004030904F0
S11381603A034600520045004500530043004100D5
S11381704C0045002000530045004D0049004300D9
S11381804F004E0044005500430054004F0052007D
S1138190200049004E0043002E0000002A03550031
S11381A053004200200043004F004D0050004F0098
S11381B05300490054004500200044004500560087
S11381C049004300450000003E034D0043005500B4
S11381D020004D0053004300200041004E004400A5
S11381E020004800490044002000470045004E009C
S11381F04500520049004300200044004500560059
S113820049004300450000002203420041004400AD
S1138210200053005400520049004E004700000063
S11382200000000000000000000000000400000046
S11382303A0000002A0000003E0000002200000076
S113824030C2FF1F34C2FF1F70C2FF1F9CC2FF1F3A
S1138250DCC2FF1F14C3FF1F00C3FF1F090400007B
S113826030C2FF1F0400000028C3FF1F01000000EC
S113827030B504E012F8014B00F8014B491ED1B1AE
S1138280C507F7D40129F5D0850701D4042904D200
S113829032F8024B20F8024B891E8B08EFD000EB1A
S11382A0830403E052F8045B40F8045BA042F9D372
S11382B0A1EB8301E3E730BD80B5134602461846BF
S11382C000E080B5FFF7D4FF002002BD10B51446CE
S11382D00A462146BDE810400123F8F7C9B8FFF764
S11382E0FEBFC046C046C046C046FFF7FBFD19E0CE
S11382F050F8041BCB0744BFA9F101035918121FFE
S11383000023042A41F8043BF9D25FEA827C0B463D
S113831004D54FF0000CA1F800C09B1CD10744BF4A
S11383200021197050F8042B002AE1D17047000095
S1138330BFFFFFFF2005000000C4FF1FE807000087
S10B834020C9FF1F000000002A
S9030411E7
